:020000040800F2
:10400000403600205DBA0008A1B90008A3B9000835
:10401000A5B90008A7B90008A9B900080000000068
:10402000000000000000000000000000ABB9000824
:10403000ADB9000800000000AFB90008B1B9000830
:104040009DBA0008A1BA0008A5BA0008A9BA0008DC
:10405000ADBA0008B1BA0008B5BA0008B9BA00088C
:10406000BDBA0008C1BA0008C5BA0008C9BA00083C
:10407000CDBA0008D1BA0008D5BA0008D9BA0008EC
:10408000DDBA0008E1BA0008277E0008E9BA000896
:10409000B3B90008F1BA0008F5BA0008BFB90008C2
:1040A000FDBA000801BB000805BB000809BB0008F9
:1040B000B7B90008BBB9000815BB000819BB000858
:1040C0001DBB000821BB000825BB000829BB000858
:1040D0002DBB000831BB000835BB000839BB000808
:1040E0003DBB000841BB000845BB000849BB0008B8
:1040F0004DBB000851BB000855BB000859BB000868
:104100005DBB000861BB000865BB000869BB000817
:104110006DBB000871BB000875BB000879BB0008C7
:104120007DBB000881BB000885BB000889BB000877
:1041300038B901EBC100052190FBF1F000F5A0704A
:1041400006E001EB8100A0F5C860092190FBF1F0C9
:1041500000B2704710B5DFF8144C00206060A06119
:1041600002F0E1F8012804BF082002F0C9FA01209A
:1041700002F0C6FADFF8F80BC0690A214843606113
:1041800010BD00B585B050B102F06CFB024692A1A3
:1041900000F03DF800A9422001F0C1F90AE002F068
:1041A00061FB02468DA100F032F8002200A9002038
:1041B00000F0E8FD05B000BDF0B583B004460A4646
:1041C00087A100F024F800A803F032F8DFF8A01B64
:1041D000896A00290CBF4321452100AD82B25155A7
:1041E000461CC0F10400471EB6B2042E07D220229E
:1041F000BFB2394600A8301803F046F8BE19B6B26F
:104200000020705500A9204600F078FDF7BD00A8F9
:1042100003F095B810B5002100220123934003401C
:104220005400042AB9BFC4F10704A340E41FE340CB
:104230005918C9B2521C082AEFDB084610BD2DE9F7
:10424000F54F81B05FEA0308DFF8289B09F5D076C7
:10425000DFF8240B0BD102782AB9002700240122B1
:10426000027047700DE0D9F8A071F46810E0B8F161
:10427000010F0BD1427832B90027002402700122CD
:104280004270877004E07768346901E0B768746948
:1042900000259DF80800484340000090DFF8DCAAA4
:1042A00008E00198285CFFF7B5FF05EB0A0181F8EB
:1042B000D8006D1C00988542F3D300219DF80800BA
:1042C00003E09DF8082001EB4201009A91422FD2B1
:1042D00000250AE029F81CE039F81CC04FEA1C2E22
:1042E00082F8D8E083F8D8C06D1C8542E9D20A185C
:1042F000AA1802EB0A0301EB050C0CEB0A0292F878
:10430000D8E093F8D8B04BEA0E2E29F81CE0B8F1AB
:10431000010F06D1002F14BF2EFA07FE0EFA04FE7D
:10432000D8E7002C0CBF0EFA07FE2EFA04FED1E7E8
:10433000002508E005EB0A0B9BF8D800FFF76AFFA1
:104340008BF8D8006D1C00988542F3D31CB9102F50
:1043500009D100271024641EB8F1000F05D1F460C4
:10436000C9F8A07108E07F1CF6E7B8F1010F07BF9C
:1043700077603461B7607461BDE8F78F10B582B0C3
:10438000DFF8FC4920780FF25C0120B9009110237E
:104390006022002107E06268012808D10092102302
:1043A00060220021002003F09BF860600CE00228EE
:1043B00008BF009102D0032806D10092102360228A
:1043C0000021002003F08CF82078401CC0B20428A3
:1043D00008BF0020207013BD25663A0025665600F0
:1043E0002564000000806010080464940404B44C48
:1043F00004848484848484040404040404048444BD
:104400002464A42424242424242424E40408106000
:10441000800000000000806010080484C4E4E4E42C
:10442000E4C484040404040404040404040404042C
:1044300004040404040484C4E4E4E4E4C48408102C
:104440006080000000071820408082818082828581
:1044500085888F8888888F858585858585858D95D4
:10446000A7B0AFA0A0A0A0A0A0A0A0BF804020188F
:104470000700000000000718204080848C9C9C9C52
:104480009F8F8783838383838383838383838383D0
:10449000838383838383878F9F9C9C9C8C84402011
:1044A0001807000000806010080464940404B44CF1
:1044B00004848484848484040404040404048444FC
:1044C0002464A42424242424242424E40408106040
:1044D00080000000000000F8F8808080F800804034
:1044E000404040800080404040408000004040F814
:1044F00040400000D000408040404080008040406C
:1045000040800000000718204080828180828285E0
:1045100085888F8888888F858585858585858D9513
:10452000A7B0AFA0A0A0A0A0A0A0A0BF80402018CE
:10453000070000000000001F1F0101011F000F12F3
:104540001212120B000C121212120F100000000FA8
:10455000100800001F00001F0000001F004788888F
:10456000887F000000E0F010102000008080808034
:1045700000008080F08080008080F0808000A000BB
:1045800080008080808000000080808080000000AB
:10459000000000000000806010080484C4E4E4E42B
:1045A000E4C48404040404040404040404040404AB
:1045B00004040404040484C4E4E4E4E4C4840810AB
:1045C00060800000000811111F0E000F121212125D
:1045D0000B0000000F10080000000F1008001F0063
:1045E000001F000000001F004F909090907F00007F
:1045F0000000000000000718204080848C9C9C9CD8
:104600009F8F87838383838383838383838383834E
:10461000838383838383878F9F9C9C9C8C8440208F
:1046200018070000F8B50C468578303DEDB20A2D2C
:1046300038BF2A46C578303DEDB20A2D38BF2B462B
:1046400000783038C0B20A2838BF01460026DFF8AB
:104650002C5718200FF2780700FB016C1CF807C0DC
:1046600006EB050E8EF860C000FB026C1CF807C05C
:104670008EF890C000FB036C1CF807C08EF8A8C031
:10468000761C182EE8DB102744B902230C220821DF
:104690002846FFF7D4FD05F1D80000E028460026A3
:1046A000009010230C2200210C20704300F0AAFF80
:1046B000761C082EF4DB7F1EE6D13CB901F0EDF943
:1046C00002F0B6FFBDE8F14001F0ABBFF1BD000064
:1046D00000E010080810E00000000000000F1020AB
:1046E00020100F0000000000001010F80000000073
:1046F000000000000020203F2020000000000000FB
:1047000000700808088870000000000000302824AD
:104710002221300000000000003008888848300066
:10472000000000000018202020110E0000000000F2
:104730000000C02010F80000000000000007042462
:10474000243F24000000000000F8088888080800C2
:10475000000000000019212020110E0000000000C0
:1047600000E010888818000000000000000F1120F1
:1047700020110E000000000000380808C8380800AA
:10478000000000000000003F0000000000000000EA
:10479000007088080888700000000000001C2221BA
:1047A00021221C000000000000E010080810E000BA
:1047B000000000000000312222110F000000000064
:1047C0000000000000000000000000000030300089
:1047D00000000000000000002DE9FE430E460FF22D
:1047E000F018024600F0BFF801F03EF8DFF880450F
:1047F000A16A00290CBF4321452101AD82B2515568
:10480000411CC0F10300401E8FB2032F08D22022AA
:104810001FFA80F9494601A8381802F035FD4F44C7
:10482000B9B20020485501A900F0BCFEDFF8C87DF0
:104830003878411C39700FF2640101EB401000F030
:104840008DF8292002F04CFE3878032804BF0020A0
:104850003870324600F087F801F006F8A16A0029A6
:104860000CBF4321452182B25155441CC0F10400C4
:10487000461EA4B2042C07D22022B6B2314601A8AB
:10488000201802F001FD3419A4B20020605501A9DE
:10489000382000F087FEBDE8F7830000000030609C
:1048A000C080000000000000000000000000180CA4
:1048B000060301000000000000000000000030605E
:1048C000C0803060C0800000000000000000180CB4
:1048D0000603190C06030100000000000000306010
:1048E000C0803060C0803060C08000000000180CC4
:1048F0000603190C0603190C06030100000018300A
:1049000060C08000000000000000000000000C06F5
:10491000030100000000000000000000000018304B
:1049200060C0983060C080000000000000000C06ED
:1049300003010C0603010000000000000000183015
:1049400060C0983060C0983060C0800000000C06E5
:1049500003010C0603010C06030100000090102364
:10496000102200217047414601A802F0E8BC38B58A
:10497000DFF8885C01F0D4FC022808D00ED30428AC
:104980000AD006D3052808BF0FF2480406E02C46DB
:1049900004E0DFF86C4C01E00FF2C40405F18C0078
:1049A00001F0CDFA0225142000FB054001F0C0FA09
:1049B000684300F027FE6D1C092DF4DB4FF4FA70FC
:1049C00002F076FF50211020BDE8344002F0DBBD3C
:1049D0002564000001FF0100000000000000101F1E
:1049E000101010101018040000C02010101010201B
:1049F000C0000007081010101008070010F0001089
:104A0000F01000F0100000031C0300031C03000062
:104A10000020202020202020200000000000000096
:104A20000000000001077980008079070100000084
:104A300000071C070000000000C02010101010200C
:104A4000C000000708101010100807000000101028
:104A5000FE1010100000000000000F1010080000F1
:104A600001FF4140404041FF0100101F10000000C5
:104A7000101F100000001013F300000000000000E1
:104A800010101F10100000000000E010101010F0B7
:104A9000100000609D8A8A8A8A91700001FF2010B0
:104AA000101010E00000101F10000000101F100078
:104AB00000202020202020202000000000000000F6
:104AC00000000000010779800080790701000000E4
:104AD00000071C070000000000001010FE1010105E
:104AE0000000000000000F10100800002DE9F04148
:104AF0001318DFF88882A0498D785DB90125CD7043
:104B000000250D7108254D7100250D704D70012592
:104B10008D7028E0CD7825BB0E794F7906EB000E1D
:104B2000AE449EF833E005EB080484F8D8E002EBCD
:104B3000050EC644F4182C1994F833408EF8D8406A
:104B40006D1CEDB2AF42E9D27D1C4D71761E0E7127
:104B5000EDB20B2D05D10A2048710020087101200B
:104B600025E00D7925BB0125CE784F7911E006EBC4
:104B7000050EC6442C1894F833408EF8D84006EB46
:104B8000020EAE44C644EC1894F833408EF8D84078
:104B90006D1CEDB2BD42EAD3781E4871721CCA701A
:104BA000C0B228B901204871092008710020C870DE
:104BB000BDE8F081F8B504460D46DFF89C6C142181
:104BC000304603F0A3F90FF2740724B900230A2238
:104BD0000121384606E0012C07D101230A220121D8
:104BE00007F12000FFF72BFB06E0022C04D10A227C
:104BF00001213846FFF77AFF00960A230A22062190
:104C0000562002F06DFC0FF2DC0401F075FD042863
:104C100003D104F10C00009005E0002D06BF07F160
:104C20001400009000940A2306220621502002F06E
:104C300057FC0120BDE8F240FFF7A3BA10188CC65C
:104C40006363C68C1810426331180C0C1831634230
:104C500000F01E1FF00000FF8080FF0042C68C188D
:104C60003030188CC64208183163C6C66331180844
:104C70008C8CC6C68C8CC6C68C8C313118183131E0
:104C800018183131008C8C8C8C8C8C8C8C8C8C8C8E
:104C90008C8C8C0000313131313131313131313155
:104CA0003131310080C0603098CC66333366CC98A7
:104CB0003060C08088CC6633190C060303060C19DB
:104CC0003366CC88113366CC983060C0C0603098B1
:104CD000CC6633110103060C193366CCCC6633194C
:104CE0000C06030100F0FEFFF000007F7F7F7F00D5
:104CF000FF0FE1E00FFFFF80BFBF80FFF0B583B083
:104D00000C460501DFF8786D16E03638C0B2102782
:104D1000FFB2C7F110011022019201EBD1714910CD
:104D200001EB40108019009010233A460021E8B2B0
:104D300002F0FFFB7D19ADB22078A8B114F8010B89
:104D4000202808BF0A20E3D02D2808BF0C20DFD080
:104D5000A0F130010A2903D23038C0B20E27D7E7BC
:104D6000A0F141010629D0D3F7BD0000A0310020F9
:104D70007006002010040020810800202802002076
:104D80000432002038B505460C46A2B92078A8B1F7
:104D900014F8010B2038C0B20FF2240100F058FBC8
:104DA0006D1CF3E714F8010B3038C0B20FF200614C
:104DB00000F04EFB6D1C20780028F3D131BD0000BF
:104DC00000000000000000000000000000000000E3
:104DD000000070F8F87000000000000D0D000000E9
:104DE00000383800003838000000000000000000E3
:104DF0000020F8F820F8F82000020F0F020F0F0231
:104E0000003078CE8E18100000040C38390F0600E0
:104E1000183C24BCD86030000006030D1E121E0C86
:104E200000B0F8487830000000070F0809070F09A4
:104E30000000003838000000000000000000000002
:104E40000000C0F0380800000000071F38200000F4
:104E500000000838F0C00000000020381F070000E4
:104E60000080A0E0C0E0A080000002030103020077
:104E7000008080E0E080800000000003030000006C
:104E800000000000000000000000002C3C1C00009E
:104E90000080808080808000000000000000000012
:104EA00000000000000000000000000C0C0C0000DE
:104EB00000000080E078180000181E0701000000C4
:104EC0000000F0F80868F8F00000070F0B080F0763
:104ED00000202030F8F80000000000000F0F000054
:104EE0000030380888F87000000C0E0B0908080024
:104EF0000030388888F8700000060E08080F070098
:104F00000000F8F800E0E00000030302020F0F02C7
:104F100000F8F88888880800000808080C070300D3
:104F200000C0E07858C8800000070F08080F07008D
:104F300000080888E878180000000E0F0100000043
:104F40000070F8C888F8700000070F08090F070004
:104F500000F0F80808F8F0000000090D0F03010048
:104F600000000060606000000000000C0C0C0000FD
:104F700000000060606000000000002C3C1C00008D
:104F80000080C0603018080000000103060C080013
:104F9000004040404040400000010101010101008B
:104FA0000008183060C0800000080C0603010000F3
:104FB00000303888C87830000000000D0D00000077
:104FC000F0F80888C848F8F0070F08090B0A0B0B1F
:104FD00000E0F01818F0E000000F0F01010F0F00C3
:104FE00000F8F88888F87000000F0F08080F070015
:104FF00000F0F8080838300000070F08080E060017
:1050000000F8F80818F0E000000F0F080C07030084
:1050100000F8F88888880800000F0F0808080800C2
:1050200000F8F88888880800000F0F0000000000D2
:1050300000F0F8080838300000070F08090F0F00CB
:1050400000F8F88080F8F800000F0F00000F0F0044
:10505000000008F8F80800000000080F0F08000022
:105060000000000000F8F80000060E08080F070016
:1050700000F8F880E0781800000F0F00030F0C0014
:1050800000F8F80000000000000F0F0808080800F2
:1050900000F8F820C020F8F8000F0F0001000F0FF3
:1050A00000F8F860C080F8F8000F0F0000010F0F43
:1050B00000F0F80808F8F00000070F08080F0700D4
:1050C00000F8F88888F87000000F0F00000000005A
:1050D00000F0F80808F8F00000070F08183F270054
:1050E00000F8F88888F87000000F0F00010F0E001C
:1050F000003078C88818100000040C08090F06005A
:10510000000808F8F80808000000000F0F00000071
:1051100000F8F80000F8F80000070F08080F070073
:1051200000F8F80000F8F8000003070C0C07030073
:1051300000F8F800C000F8F800010F0E010E0F0192
:10514000001838E0C0381800000E0F00010F0E00E4
:105150000078F88080F878000000000F0F00000051
:1051600000080888C8783800000E0F0908080800F1
:105170000000F8F80808000000007F7F40400000B1
:10518000001878E08000000000000001071E1800F1
:1051900000000808F8F80000000040407F7F000091
:1051A00030180818302030180000000000000000FF
:1051B00000000000000000004040404040404040EF
:1051C000000002060E0800000000000000000000C1
:1051D0000000202020E0C00000060F09090F0F008A
:1051E00000F8F82020E0C000000F0F08080F0700AB
:1051F00000C0E0202060400000070F08080C0400F9
:1052000000C0E02020F8F80000070F08080F0F008A
:1052100000C0E02020E0C00000070F0909090100DC
:105220000080F0F88888880000000F0F0000000060
:1052300000C0E02020E0E00000474F48487F3F00EA
:1052400000F8F82020E0C000000F0F00000F0F0052
:10525000002020ECEC0000000008080F0F080800F8
:1052600000002020ECEC0000004040407F3F0000A8
:1052700000F8F80080E06000000F0F01030E0C0042
:10528000000808F8F80000000008080F0F080800E0
:1052900000E0E020E020E0C0000F0F0007000F0F4B
:1052A00000E0E02020E0C000000F0F00000F0F0022
:1052B00000C0E02020E0C00000070F08080F070032
:1052C00000E0E02020E0C000007F7F08080F07001A
:1052D00000C0E02020E0E00000070F08087F7F000A
:1052E00000E0E08040606000000F0F000000000060
:1052F00000C0E0202020200000080909090F060056
:105300000020F8F8202020000000070F08080800FF
:1053100000E0E00000E0E00000070F08080F0F00C9
:1053200000E0E00000E0E0000003070C0C070300D1
:1053300000E0E000C000E0E000030F0C030C0F03EE
:105340000060E08080E06000000C0E03030E0C00A3
:1053500000E0E00000E0E00040474F68381F070031
:1053600000202020A0E06000000C0E0B09080800BF
:105370001C14DCE02020E0C000000F1F10101C0CEB
:1053800000000000FF00000000000000FF0000001F
:105390001C141CE0E02020200000001F1F01010061
:1053A00000060101020204040000000000000000E9
:1053B0000000F0F80868F8F00C00070F0B080F0762
:1053C0000000202030F8F8000C000000000F0F0053
:1053D000000030380888F8700C000C0E0B09080823
:1053E000000030388888F8700C00060E08080F0797
:1053F000000000F8F800E0E00C00030302020F0FC9
:105400000000F8F8888888080C000808080C0703D2
:105410000000C0E07858C8800C00070F08080F078C
:105420000000080888E878180C00000E0F01000042
:10543000000070F8C888F8700C00070F08090F0703
:105440000000F0F80808F8F00C0000090D0F030147
:1054500001EB00100090102308220021E800C0B2E8
:1054600002F03EB810231022002102F039B838B5FE
:105470000FF6980451EA000213D100250CE0012D2B
:1054800005D1009400F046F802F02AF804466D1C9D
:10549000022D3DDA002DF2D10094FFF760FA0846A4
:1054A000F2E7C8B1002933D101280AD104F1200064
:1054B000009010231022502002F012F804F1400056
:1054C00015E0022824D1009410231022002002F0BD
:1054D00007F804F1600017E0D1B101290DD104F102
:1054E000200000F016F801F0FBFF04F180000090AE
:1054F00010231A460021084608E0022908D100942A
:10550000FFF7B0FF04F1A00000F003F801F0E8FF9E
:1055100031BD00901023102200215020704770B53B
:1055200082B004460D460FF22C060EE015F8010B72
:105530002E38C0B2062101FB006000900523062230
:105540000021E0B201F0CCFFA41D28780028EDD1A5
:1055500073BD0000000000100000101010101010AB
:10556000001F1115111F0000111F1000001D15153F
:10557000151700151515151F000F08081F0800172F
:105580001515151D001F1515151D00010101011F21
:10559000001F1515151F00171515151F00070810FA
:1055A00008070000F8B504460D460026DFF85479D8
:1055B0000DE0142101FB0070009010230A2200214D
:1055C000F6B20A2000FB064000F01CF8761C287892
:1055D00088B115F8010B432808BF0B20E9D04528F6
:1055E00008BF0C20E5D0A0F130010A293ABF3038BD
:1055F000C0B20A20DDE7F1BD3D320020B8610008ED
:1056000064620008C0B201F06BBF00002DE9F04FEA
:1056100089B004468846914601A8142102F076FC20
:105620000020ADF800000022DFF8DC0850F824105C
:105630001046FFF7A7FB4FF00A0A80A7DFF8CC5807
:105640000A2C51D8DFE804F006080C11131D2F3B7B
:1056500041504B00686900E0286990FBFAF209E0CC
:10566000E8696421B0FBF1F204E02A6A02E0A8696B
:10567000B0FBFAF23946FFF777F900F0F5F8064685
:1056800032E0E86AB0FBFAF23946FFF76DF9E86AF2
:10569000B0FBFAF10AFB11023946FEF7B8FD00F043
:1056A000E3F8461C20E0A86A002807BF032264A193
:1056B000032264A101A802F03DFC022614E0686AFE
:1056C000002814BF60A061A004E0686B00280CBF34
:1056D0005FA060A001A902680A60032604E00FF63B
:1056E0006C0101A801F02BFEF01D8DF8020006F1FF
:1056F00008070FF2681BDFF81868B9F1010F3CD1F9
:10570000B069B0F5167F35D298F8000054A1012891
:1057100006D100220720FFF735FB002259460BE097
:105720000FF24019022806BF002259460022072026
:10573000FFF728FB00224946F8B2FFF723FB052CB0
:1057400006D100F094F8012200A99DF8020002E0C1
:10575000002201A90820FFF715FBB069002869D1D4
:105760004FF47A70B061B8F1000F63D0002088F870
:1057700000005FE000F080F857E0092C3DD1B069EF
:10578000002857D100F0AFFE044600F0F5FE07B246
:1057900024B22146A86A0128384612D101F0A7FD9B
:1057A00032280BD2394600F07DF90546214600F03B
:1057B00079F995FBFAF20FF2A4710AE00FF2A471E5
:1057C0000DE001F094FD322807D297FBFAF20FF2B8
:1057D0009C7106A801F0B3FD04E00FF2987106A8D1
:1057E00001F0ADFD002206A90720FFF7CBFA00204B
:1057F000FEF7C7FCC820B0611CE00A2C05D10022CE
:1058000001A90020FFF7BEFA14E000F035F8052CDE
:1058100006D100F02CF8012200A99DF8020002E058
:10582000002201A90820FFF7ADFA0022CCA1F8B2AE
:10583000FFF7A8FA09B0BDE8F08F0000256400006A
:10584000207B0000207D0000204C480020524800B2
:105850004F464600204F4E0000030020200000006D
:105860003C0000003E00000001A801F0E1BC002265
:1058700001A90820FFF786BA002259460720FFF742
:1058800081BA00002DE9F84F044600208DF8000091
:10589000DFF87C6600F0FAF8DFF878B6DFF86C76AF
:1058A0000A2C0CD8DFE804F0065D6366696C6F7241
:1058B0007578A70007F11405B869CBF8080000F067
:1058C000E5F84FF4967001F0F3FF0C20604350F8B8
:1058D0000B805844D0F80490B0F808A0B86A0128AA
:1058E00009D1002C18BF012C05D1DBF86C80DBF846
:1058F0007090BBF874A000F0C5F800F0FCFC002824
:1059000000F0B28029680A46B0F5014F18BFB0F523
:10591000807F79D18945BEBFA1EB0A01494549463F
:1059200029608A426ED0062C68D100296AD1796933
:1059300009B20120FEF7FCFB8346396909B2012058
:10594000FEF7F6FB3861BBF57A7FB8BF4FF47A7B80
:10595000C7F814B0B0F57A7F54DA4FF47A70386132
:1059600050E007F11005B869CBF81400A7E707F17C
:105970001C05A4E707F12005A1E707F118059EE73C
:1059800007F12C059BE707F1280598E707F12405A7
:1059900095E707F1340592E701F04AFE00F041FE79
:1059A00000F0D6FD00F0A4FC012807D1DFF868055F
:1059B0000068386302F0EBFA02F01AFDDFF85C458C
:1059C0002078002859D0012807BF00220FF2AC51DF
:1059D00000220FF2B4510020FFF7D4F900F021FEAD
:1059E00000F05BF800F01DFE00F057F8002020707A
:1059F00001F01EFE41E003F094F83EE0072C08BFE2
:105A000001F0E8FD012022E040281CBF48F24003DD
:105A100098421ED1414505DA0AEB01004146804516
:105A2000C8BF014629608A4210D0062C0AD101293C
:105A30000CD1796900F035F87861396900F031F8F6
:105A4000386103E0072C08BF01F0C4FD02208DF887
:105A50000000322001F02CFF4FF47A60F0604FF428
:105A6000C870B06100F00EF800F0DBFDF0680028AF
:105A70007FF441AF4FF4FA50F060BDE8F18F0000C1
:105A8000985F0008012200A92046BFE54FF47A7014
:105A9000B0614FF47A60F06070474FF47A7001F0B3
:105AA00007BF09B20020FEF743BB70B500250026F2
:105AB00001F0BEFD2A4611460846FFF7A7FDDFF8B4
:105AC000504442F21070E06000F015FCB0F140016B
:105AD0000ED0C03906D047F64072891A18D0C039A6
:105AE0000DD01AE0F6B2002E0CBF0A26761E0DE08D
:105AF000F6B20A2E38BF761C08D3002606E000F066
:105B000004FCF0B2FFF7BEFE00F02CF8002505E023
:105B100000F0FBFB0020E06070BD30B101F088FDBB
:105B20004FF4FA50E06000F01DF800F07AFD0A2012
:105B300001F0BEFEA06908B900F014F8A06858B9D9
:105B4000282D09D20DB900F0EAFD462001F0A3FE90
:105B50004FF4FA70A0606D1C282DB5D170BD000007
:105B60002020200000220021F0B24FE570B582B065
:105B7000044650250E01F6B20EE0102105F110008A
:105B800001F001FD0094FEF7EAFEE8B201F0A8FC86
:105B9000103D192001F08CFEB542EEDA73BD2DE9FF
:105BA000F04182B00A24D948B0F9142092FBF4F5F0
:105BB0002DB2642695FBF6F2D2B206FB125393FB8C
:105BC000F4F3DBB206FB125504FB1355EDB2D44CD3
:105BD0002678012E03D1A6600026E66006E0022E9C
:105BE00005D10026A6601026E66000262670002754
:105BF0000FF2A43602E08CF838E17F1CDFF824C3F2
:105C0000B7EB410F20DA06EB421E17F80EE007EB68
:105C10000C0888F8D8E006EB431E17F80EE088F869
:105C2000F8E006EB451E17F80EE088F818E1D0F80A
:105C300028E0BEF1010FBC4407EB060E0CBF9EF836
:105C4000E0E19EF8A0E1D6E767600CF1D800012101
:105C50006160FEF783FE60680007000E01F040FC03
:105C60006168491C61600529F3DBA068E16850EABE
:105C7000010202D019B9102804D1002005E0481E05
:105C8000E06001E0401CA0600120BDE8F6812DE944
:105C9000F8439E4CB4F914900FF270050021284689
:105CA000FFF764FF4FF47A7699FBF6F7FFB20FF235
:105CB000E828012108EB4710FFF758FF06FB17996A
:105CC000642699FBF6F7FFB2022108EB4710FFF7B5
:105CD0004DFF032106FB17900A2290FBF2F0C0B2A1
:105CE00008EB4010FFF742FFA06A012807BF04211C
:105CF00008F5F070042108F5D070FFF737FF052193
:105D000005F12000BDE8F44330E70000808040400A
:105D10002020101008080404FE000000000001010B
:105D200002020404080810103F0000000000FE04F6
:105D300004080810102020404080800000003F1020
:105D4000100808040402020101000000008080C065
:105D5000C06060303018180C0CFE00000001010318
:105D60000306060C0C181830307F00000000FE0CF3
:105D70000C181830306060C0C080800000007F3098
:105D80003018180C0C060603030101008080C0C007
:105D9000E0E0F0F0F8F8FCFCFE000000000001017B
:105DA000030307070F0F1F1F3F0000000000FEFC4A
:105DB000FCF8F8F0F0E0E0C0C080800000003F1F79
:105DC0001F0F0F07070303010100000070B54F4AC2
:105DD000B2F914204FF47A7392FBF3F4642592FB2A
:105DE000F5F6B6B249B9801890FBF5F190FBF3F0E7
:105DF00080B2A4B2A04209D10AE0101A90FBF5F1DA
:105E000090FBF3F080B2A4B2A04201D0032070BD99
:105E100089B2B14201D0022070BD012070BD2DE9D0
:105E2000FC4D3A4CA5693B48A16A002907BF0668AA
:105E3000D0F804B0C66ED0F870B001F0F9FBFFF7EF
:105E400026FFDFF8CC8042F21070C8F80C00ADB22B
:105E50004FF47A6A324F29E040281CBF48F24001D3
:105E6000884221D16069B04219DA012038700021DE
:105E70002846FFF7ABFF6169691861618E42D8BFA0
:105E8000314600F051F8022038700021FFF7EFFA98
:105E90006069B04203D102210020FFF7E8FA322006
:105EA00001F006FDC8F80CA000F0BBFBD8F80C0010
:105EB00030B300F020FAB0F5807F18BFB0F5014F85
:105EC000CAD160698345EDDA012038700121284686
:105ED000FFF77CFF6169491B61615945B8BF5946AD
:105EE00000F022F80220387000210120FFF7BFFAED
:105EF00060695845D6D101210020FFF7B8FAD1E7F3
:105F0000BDE8F38DE8B400084407002070060020C7
:105F1000A0310020C80500203008002028080020FB
:105F2000640800202802002061610022102136E66A
:105F30002838009010230A2200210A207047009080
:105F4000102310220021084601F0CABA526573746A
:105F50006F72652044464C540000000025647D208B
:105F6000000000002D2D7D200000000025647B2016
:105F7000000000002D2D7B2000000000436F6D709D
:105F80006C657465642E00005265747279206C61D2
:105F90007465722E00000000000000E0F8180C0C80
:105FA0000C8CCC78F8E000000000001F7F78CCC695
:105FB000C3C1C0607F1F000000000000303038FC0B
:105FC000FC0000000000000000000000C0C0C0FF96
:105FD000FFC0C0C00000000000000070781C0C0C66
:105FE0000C0C8CDCF8700000000000C0E0F0F8DC65
:105FF000CEC7C3C1C0C0000000000070781C0C0CEC
:106000000C0C0C9CF8F000000000003878E0C3C3D2
:10601000C3C3C3E77D3800000000000080C0E0700B
:10602000381CFCFC000000000000000F0F0D0C0CE1
:106030000C0CFFFF0C0C0000000000FCFC8C8C8C96
:106040008C8C8C8C0C0C00000000003171E1C1C103
:10605000C1C1C1E37F3E000000000000C0E0703815
:106060001C0C0C0C000000000000003F7FE7C3C3C5
:10607000C3C3C3E77E3C00000000000C0C0C0C0CFA
:106080000C0CCCFC3C0C0000000000000000C0F038
:106090003C0F03000000000000000000F0F89C0C22
:1060A0000C0C9CF8F00000000000003C7EE7C3C32D
:1060B000C3C3C3E77E3C0000000000F0F89C0C0C5A
:1060C0000C0C0C9CF8F000000000000001C3C3C3DE
:1060D000E3733B1F0F0300000000000000000000FE
:1060E00000000000000000000000000000000000B0
:1060F00000000000000000000000000000000000A0
:10610000F000000000000000000001010101010199
:106110001F0101010101010000000000000000005A
:106120000000000000000000000101010101010168
:1061300001010101010101000038283880C06060C0
:106140006060604080000000000000001F3F606051
:106150006060602010000000000000000000C0C06F
:10616000C0C000000000000000000000000030304F
:1061700030300000000000000038283800FCFC8CA3
:106180008C8C8C8C8C00000000000000007F7F0154
:106190000101010101000000FCFC0000000000C042
:1061A000C00000000000FCFC7F7F30180C060301DB
:1061B0000103060C18307F7F01FF00E11FE000FFA4
:1061C000010000011E0100011E010000006010100E
:1061D0009090E0000000000E111110081F18000040
:1061E0001010F04020101030000010101F10100090
:1061F0000000000010F02010101010E00000101F30
:1062000010000000101F100000001013F300000029
:106210000000000010101F101000000010F02010EF
:10622000101010E00000101F10000000101F1000E0
:1062300000E010101010F0100000007D8A8A8A8A99
:106240009170000000000080E0F8FE0707FEF8E013
:1062500080000000101C1F1F1F1F1F12121F1F1F76
:106260001F1F1C10001C2221414141820700001EFB
:10627000081010101008070000C0A090909090A087
:10628000C0000007081010101008040010F02010C3
:10629000101010E00000101F10000000101F100070
:1062A00000202020202020202000000000000000EE
:1062B0000000000001FF21212121F9030400101F2B
:1062C0001010101010180400001010F040201010D2
:1062D00030000010101F101000000000001010F01F
:1062E0004020101030000010101F1010000000009F
:1062F000B84800787047B849086900220A617047B9
:1063000000B10120B4490870704710B5B24C0020AC
:1063100020702061322001F0CBFA0120207010BDE6
:10632000AC484078704780B500F09CFA0A21A94A31
:10633000D3684B43834203D204205070012002BD36
:1063400013695943884209D25088401C508080B25A
:106350000B2824BF05205070022002BD0020508071
:1063600001205070002002BD2DE9F0419B490868D2
:10637000C0430968C94301F00201974A5378147871
:106380002340537094781578254095709488C607FB
:1063900002D500261681641CD688022902D1002766
:1063A0001781761C48F2400C4FF4014E8C4FA4B27A
:1063B000192C12D392F80080B8F1000F18BF002BEF
:1063C0000BD0B6B24EB97B6A002B14BFC2F810E0F6
:1063D000C2F810C00123538111E0B6B2192E0ED3BA
:1063E0001378002B18BF002D09D044B97B6A002B0D
:1063F00014BFC2F810C0C2F810E0012393814FF41B
:106400008073C00714D4508960B9192C06D22CB1FE
:10641000786A002812BF1361402010611089401C67
:10642000108101E0002050810CB90120507000243F
:106430009480A1B9908960B9192E06D22EB1786ADC
:1064400000281ABF4020106113611089401C108180
:1064500001E0002090810EB9012090700026D680C6
:10646000BDE8F08170B55F494A68D3089CB2C500A9
:106470000E781EB94D600120087009E0844234BFD7
:10648000041B241AA4B23D2C3CBF8018C51A4D60D1
:10649000E80870BD10B5002001F0FDF95248402118
:1064A00001600A2001F006FA504C01202070022001
:1064B00001F000FA00202070606810BD4C490A7895
:1064C00022B9C000486001220A7007E04A688018BB
:1064D000931002EB5372A0EBE2004860811000EBD6
:1064E0005170C01070472DE9F04104464FF000088C
:1064F0000A27404E012001F0C9F93168411872683D
:10650000824238BF02467260B268904288BF10462D
:10651000B060012F13D17068081AB168401AC00822
:10652000FFF7CCFF05462CB940F6E4406843000B6A
:10653000A0F5FA78002141F28830B06071603160D6
:106540007F1ED7D1002C14BF28464046BDE8F081FD
:1065500010B5FFF79FFF04460020FFF7C4FF1D4959
:10656000B4F5C87F05D2B0F5967F02DA8C600120C1
:1065700000E00220087010BD38B5FFF78BFF04461D
:106580000020FFF7B0FFB0F5967FC8BF4FF49670BC
:1065900010498A68A21A122392FBF3F303F28A23AA
:1065A0004FF462756A4392FBF3F28018A4F611620D
:1065B000B2F5C77F9ABF8A88521C00228A808A88D7
:1065C000052A2CBF02220122B4F57A6FC8BF03222C
:1065D0004A7032BD280800203C080020080C014009
:1065E00070060020EC31002014080140E431002046
:1065F000F43100209408002010B5044645F25550AF
:1066000002F020FC032002F020FC0A20604340033B
:10661000000C02F01DFC02F01EFC02F021FC012027
:1066200010BD80B502F017FC012002BDDFF8D80ACA
:1066300000687047DFF8D01A0A68824205D24FF02E
:10664000FF32101A0968081870470968081A70475D
:106650002DE9F04F83B004460D460026DFF8AC7AF2
:1066600001223B4602F008FC8FBFCDE90045CDE991
:10667000006726462F4630463946DDE9002302F002
:10668000FBFB33D8DDE9000132463B4602F00CFC4F
:106690000022DFF87C3A02F07BFC804689464246C5
:1066A0004B4602F075FC82468B4622462B4602F092
:1066B00041FDDFF8602ADFF8603A02F0FBFD09D205
:1066C000DFF8582ADFF8583A02F0D6FB02D84046E5
:1066D00049460EE02046294652465B4602F0EAFD56
:1066E0002EBFCDE9008946464F46C4E70020DFF8BB
:1066F000341A03B0BDE8F08FDFF82C0A0078704739
:10670000DFF8241A0A784A700870012088707047F0
:1067100038220FF6E421DFF8140A01F0FBBB38B58C
:10672000DFF80C4ADFF80C5A012808D100F053F8C2
:106730004FF4806100F048F800F044F80FE098B999
:10674000DFF8E409C07820B100F041F84FF480612F
:1067500032E000F037F800F03AF800F040F81E2080
:10676000BDE8324001F0A4B8022813D100F033F89C
:106770004FF4807100F035F800F031F800F0AFF917
:1067800000F025F800F0ABF908212846BDE83440B8
:1067900002F00FBE032814D100F01DF84FF48071F1
:1067A00000F01FF800F01BF800F099F900F00AF86B
:1067B00000F095F94FF480712046BDE8344002F0B6
:1067C000F6BD31BD4FF48071204602F0F2BD0821C4
:1067D000284602F0ECBD0821284602F0EABD4FF43D
:1067E0008061204602F0E3BD2DE9F04100270C2432
:1067F000DFF84459DFF84469DFF834890121404665
:1068000002F0D5FD022001F053F800203070012085
:1068100001F04EF82868C7190121404602F0C9FD71
:10682000022001F045F80120307001F041F828689D
:106830003F1AFFF7F6FE641EE0D1DFF80409784343
:1068400040F22A31B0FBF1F0000BDFF8F84820608D
:106850006421B0FBF1F00B2828BFFFF7C5FF2068CB
:10686000BDE8F08138B500240A25DFF8DC0802F025
:106870009DFE04196D1EF8D10A20B4FBF0F04FF410
:10688000A5714843000B892148431B21B0FBF1F05F
:1068900032BDDFF8940800218181C18101824182EB
:1068A000016241610F2101830421418332218183EF
:1068B0007047F0B500220123DFF86C18C881B1F9E8
:1068C0000C00B1F90E40051B0D820D7900F11E067A
:1068D000A642B8BF6D1CEDB20B2D28BF0A6200F1B5
:1068E0005A07A742B8BF00258442B8BF00250D71E2
:1068F000B1F91000B0F5967F05DA01220C7914B9D0
:106900000C6A04190C62B1F90E40B1F90C50A542A1
:106910000DDA641B24B28D6E012D04D11F2C02DB15
:1069200000220A628A66972CA4BF00220A6200F144
:106930001E04A4B23D2C38BF00231F2804DBB1F98C
:106940001240041B0AD508E06FF01D04A04205DACE
:10695000B1F91240041B012C00DB00230C8B4D8B82
:106960006A430D6A6A4300FB04228C8BB1F9125012
:10697000451B6C4303FB04224882012AB8BF002256
:1069800004DBB2F5FA6FC8BF4FF4FA624A6190B205
:10699000F0BDDFF894279181884204DA091A1229A0
:1069A00004DB002105E0411A132901DA022100E08D
:1069B000012191847DE7F8B507460024002500F009
:1069C00003FC2046FFF7ABFEC82000F071FFDFF8A4
:1069D00058675FB3306DDFF86C170968484302F001
:1069E00015FEFFF735FE0022DFF8603702F0D0FA1F
:1069F00004460D4604270220FFF791FE00F06FF8D1
:106A00007F1EF8D1FFF72EFF40F2A331884202D358
:106A10000020F0700DE00120F07000F060F800F050
:106A2000D3FB0020BDE8F24079E6F1BDF078002804
:106A3000F3D11426FFF716FF143002F0E7FD2246CB
:106A40002B4602F037FC22D2FFF70CFF02F0DEFDEE
:106A500002460B462046294602F06CFB0022DFF876
:106A6000F03602F021FA02F0DFFD80B290FBF6F47E
:106A7000A4B2102C28BF0F2402D2A4B2002CD4D070
:106A80000220FFF74CFE00F02AF8641EF5E7FFF73E
:106A9000E9FE02F0BBFD02460B462046294602F005
:106AA00009FCC2D2FFF7DEFE143002F0AFFD224631
:106AB0002B4602F03FFB02F0B7FD80B290FBF6F4EC
:106AC000A4B2102C28BF0F2402D2A4B2002CACD048
:106AD0000320FFF724FE00F002F8641EF5E71E20F5
:106AE00000F0E6BE000000002DE9F04F85B04FF049
:106AF000000BDFF834466078A1780A254FF47A7AE3
:106B0000DFF850664FF4FA782278012A0CD0032A75
:106B100000F03081042A00F00682052A00F0898204
:106B2000082A00F0A582EBE288B981B100F080FD6F
:106B300000F095FD002104F13000FDF773FD58468B
:106B400000F03DFBC6F808800120A06607E0B069B0
:106B500028B9706918B1FDF711FCC6F818A0606E6D
:106B60000028B0681CD088B9E06EB0F5966F0DD2E1
:106B700008B900F029FB0020FFF7D1FD322000F01A
:106B80008AFEC6F80880E06E401CE066E06EB0F554
:106B9000966F1FD100F018FBE06E401CE06619E014
:106BA00080B9A07A3C280DD208B900F00DFB002076
:106BB000FFF7B5FD322000F06EFEC6F80880A07A1F
:106BC000401CA072A07A3C2804D100F0FDFAA07A03
:106BD000401CA072A07848B1002000F0F0FA3320E9
:106BE000A0855846E066A0720120A066FFF7FCFD74
:106BF000FFF781FB5FEA00091CBF706900280CD019
:106C0000DFF840754FF06408484640283CD0B0F5A6
:106C1000807F03D0B0F5014F3AD07FE0FFF7E4FD6D
:106C20003868B0FBF8F0801E09280ED300F000FD94
:106C300000220FF2AC511046FEF7A4F840F2DC50EF
:106C400000F036FE00F0F4FC68E04FF0050AFFF7B4
:106C500021FCB0F57A6FC8BF0BF1010BBBF1050F3A
:106C600007DBDFF8F404032101700820FFF748FD7B
:106C700002E0BAF1010AEAD10120FFF79CFE0020F0
:106C800000F021FE032000E00520FFF739FD45E07C
:106C9000FFF73BFB00F0CCFC3868002814BFB0FBCA
:106CA000F8F200220FF2445100F082FA002200A90B
:106CB0001046FEF767F800A800F0BAFA8246386876
:106CC00000281EBFB0FBF8F108FB1100002814BF1C
:106CD000B0FBF5F200220FF2980800F068FA0122EA
:106CE00000A95FFA8AF0FEF74DF8386800281ABF4D
:106CF000B0FBF5F105FB1102002200F058FA00226A
:106D000000A90AF10100C0B2FEF73CF8FFF789FCC8
:106D10004FF47A7000F0CCFDFFF783FC706990B9F6
:106D2000A08D80B1E18D491CE18589B232290AD15B
:106D3000411EA185C0B200F095FB0020E085A08D2A
:106D400008B900F0A4FB02F095FC002808BFB9F1D7
:106D5000000F0BD0E06C68437061A08D002805D156
:106D60003320A08500F07EFB00F085FBC8E100BF6A
:106D70002564000039B10020A07000F059FC58468D
:106D8000306000F01DFA207A20B100F01DFA0020DA
:106D9000FFF7C5FCFFF7C7FA08B9E0712072A06ED3
:106DA000012822D1FFF7BFFA40B1E079401CE07121
:106DB000C0B2C828DAD10020E071B2E0E071FFF77C
:106DC0009AFA814648F24001401A2CD0C03834D19A
:106DD000FFF79BFA002000F05EFD00F029FC052083
:106DE000FFF78EFC5846706027E030690028E6D136
:106DF000FFF799FA0028E2D0E079401CE071C0B2B8
:106E00000A28DCD10020E071207A401C20724FF467
:106E10007A613161C0B20328D1D10820FFF770FC3C
:106E2000002020726CE1FFF770FA002000F033FDC3
:106E30000120FFF765FC00F0C7F9616CA06D012827
:106E400003D109B2FDF774F90146218500F027FD51
:106E500030B9FFF791FB00F0A3F900B200F01BFD81
:106E600000F098F912283CBF208DE084A08CC7B2B6
:106E7000012F06BF60790128C6F808A06771B068C5
:106E8000002804BFB069002817D1A07910B90120EB
:106E900000F092F9B4F92810A06D012807D100F094
:106EA00096F900F097F99AFBF5F109B201E000F0CC
:106EB00066F900F06AF9C6F818803068C0B9B068A1
:106EC000B0B1A07908B100F076F9B4F92610618567
:106ED000A06D012802D100F07AF9608500F047F931
:106EE00002F0C8FB01463846FDF764FEC82030605A
:106EF00002F0C0FB002808BFB9F1000F01D000F07C
:106F00005FF9706920B900F0C6FC0420FFF7F8FBB8
:106F1000FFF706FA022885D3FFF702FA042880F06B
:106F2000EF800820EAE031B10020A070306000F06E
:106F300047F90120A066206CA16D012903D101B29F
:106F40000120FDF7F5F82085616C206C814208DA9C
:106F5000A06D012804D109B2FDF7EAF8208500E010
:106F60002185706848B9FFF707FB00F019F900B2F6
:106F700000F091FC4FF49670706000F00BF912284D
:106F80003CBF208DE084A08CC7B2012F06BF607982
:106F90000128C6F808A06771B068002804BFB0696E
:106FA000002816D1A07908B90120A071B4F92810E1
:106FB000A06D012807D100F00AF900F00BF99AFB47
:106FC000F5F109B201E000F0DAF800F0DEF8C6F8F9
:106FD0001880E08C60853068B8B9B068A8B1A07935
:106FE00008B100F0E8F8A06D012804D1B4F92A1026
:106FF00000F0EDF8608500F0BAF802F03BFB0146C6
:107000003846FDF7D7FDC8203060FFF789F9022820
:1070100028BF082072D202F02DFB10B9FFF76BF9E0
:1070200008B103206AE07069002869D100F033FCE0
:1070300063E0012812D1FEF738FD434C002200F036
:1070400091F800F0A4FF01F0D3F9012200F08AF8D2
:107050000120FFF755FB00F0B7F851E003284FD1AE
:10706000FEF7DDFE0320FFF74BFB0120A06647E0A3
:1070700039B10020A07000F0DBFAC6F818800120BA
:10708000A066364828B1002000F005FC34484021B5
:107090000160FFF745F901281ED020D3032804D052
:1070A00003D3052808D003D319E0FFF765FA16E0EB
:1070B000FFF739F998B90FE001250120FFF77BFCB4
:1070C000FFF7D0FB40F28B21884224BF0320FFF75B
:1070D00017FB6D1EF1D102E00320FFF711FBB06931
:1070E00070B9FDF744FCC6F81880607A401C6072E5
:1070F000C0B2032804D1002060720120FFF700FB1A
:1071000005B0BDE8F08F0000203200200000F03F05
:107110000000E03FFDA9F1D24D62503FFCA9F1D241
:107120004D6250BF0000F0BF4006002070060020F6
:1071300000080140000C0140E8310020E43100204B
:107140007064080024320020002801400000244020
:10715000000034C0A0310020290800209F780008DA
:10716000140801404FF4A071204602F0BCB9B4F9F4
:107170002A0090FBF5F109B20020FDF71DB891FB44
:10718000F5F109B2B4F92600704790FBF5F000B2B2
:10719000FDF722BBB4F92810B4F9260000F0A7B817
:1071A000E084B4F92810B4F92600FFF7F2BB414699
:1071B00000A800F0C4B80020A07100F039BAA07097
:1071C000E06C6843706170470120FFF7A8BA0020A7
:1071D000FCF7AEBF8246B4F926105846FCF7A8BFAC
:1071E0002020204E6F2054697021000054697020C7
:1071F000523A256400000000312E303700000000B4
:107200000000000000000000D0070000B80B0000E4
:107210006400000050460000120000000000000062
:107220000000000082000000660000000100000075
:1072300000F10103810704D010F8011B89B1810717
:10724000FAD10268B2F10131914311F0803F04BFDD
:1072500050F8042FF6E710F8011B11B110F8011BCC
:10726000FBE7C01A704750F8041B61B150F8042BBB
:10727000D30744BFA9F101039A18002342F8043B45
:10728000091FFAD1EFE7704762F30F2262F31F4242
:10729000401810F0030308D0C91A1FD3DB0748BFFA
:1072A00000F8012D28BF20F8022D130030B4144639
:1072B0001546103928BF20E93C00FAD8490728BFF5
:1072C00020E90C0048BF40F8042D890028BF20F8B1
:1072D000022D48BF00F8012D30BC7047C91818BFF7
:1072E00000F8012DCB0728BF00F8012D704781421F
:1072F00001DA401A7047081A704770B5002200285A
:1073000003D52D220A70012240420A2390FBF3F498
:10731000012502E094FBF3F45D43002CFAD155B152
:1073200090FBF5F404F130065654521C05FB140092
:1073300095FBF3F5F3E700205054084670BD0CB4FC
:107340002DE9F04383B004460D4600270026002CAB
:1073500000F083800DF128084FF00A0903E0795D01
:10736000315506467F1C795D002973D0701C252994
:10737000F5D17F1C795D632906D0642914D0662974
:1073800021D0732905D0EAE708F1040818F8041C95
:10739000E6E758F8040B00210A5C002A1EBF3255AC
:1073A000491C761CF8D1DDE700A958F8040BFFF75B
:1073B000A4FF002100A8085C00281EBF3055491C0E
:1073C000761CF7D1CEE758F8040B411E092924BFDB
:1073D000A0F10A015A29C5D3A0F16401B1F5617F7A
:1073E00015D290FBF9F109FB11003030E07091FBF0
:1073F000F9F009FB10113031A1702E21617090FB62
:10740000F9F109FB1100303020700426AAE7A0F53D
:107410007A7142F228329142A4D290FBF9F109FB31
:1074200011003030207191FBF9F009FB101130315F
:10743000E1702E21A170014691FBF9F009FB1011BA
:107440003031617090FBF9F109FB11003030207090
:10745000052687E7002030552046BDE8FE035DF88D
:107460000CFB000010B504463C21812002F067FAB5
:107470003C21204630E080B53C218D2002F05FFAAF
:107480003C21142002F05BFA3C21AF200AE080B5D9
:107490003C218D2002F053FA3C21102002F04FFADB
:1074A0003C21AE20BDE8044002F049BA10B50446C4
:1074B00008465B49496A01B120343C215038C0B2CA
:1074C00002F03DFA3C21E4B2200940F0100002F045
:1074D00036FA3C2104F00F00BDE8104002F02FBA4C
:1074E0002DE9F041044690465818C0B2CE08072254
:1074F000114218BF761C811000EB5171CA10B0EB1D
:10750000C2011ABF501CC5B2D5B2069F0BE031466E
:107510002046FFF7CBFF01233C224146384602F0CC
:10752000F5F94744761CF6B2AE42F0DB3846BDE8CA
:10753000F0812DE9F843804691465818C0B2CF0833
:107540000722114218BF7F1C811000EB5171CA1035
:10755000B0EBC2011ABF501CC6B2D6B2089D099C3E
:107560000BE039464046FFF7A1FF01233C22494684
:10757000284602F0CBF965197F1CFFB2B742F0DB59
:107580002846BDE8F28330B5A1B004460D4601A8F7
:1075900000F0BCFC00F05FF82A460021E0B2FFF7E3
:1075A0009FFF00F058F82A460821E0B2FFF798FF45
:1075B00021B030BD80B54FF40040ADF8000003208D
:1075C0008DF8020010208DF8030000A9154801F085
:1075D00089FE01BD10B5144C4FF40041204601F066
:1075E000E8FE022000F064F94FF40041204601F06B
:1075F000DEFE022000F05CF90C480949496A19B91D
:10760000C8214171A12102E0C0214171A021417234
:1076100000233C221721BDE8104002F077B900009A
:1076200070060020000C01400008014010080020F6
:1076300000B5A1B0802101A800F068FC00F00BF8B3
:10764000802200F0B9F800F006F88022194600F018
:10765000B4F821B000BD01A80090082370472DE9BF
:10766000F041A2B00125802102A800F04FFC0022C9
:1076700001A90FF24C1000F0AAFC040000F07F807A
:107680002078422804BF60784D2840F0878094F825
:107690003600FF2804BF94F83700FF2804D194F87F
:1076A0003800FF2808BF002500F081F801260F27C9
:1076B000002000210C2202FB0712121992F83E2032
:1076C00080234FF0080C03EA020E1DB1BEF1000F3B
:1076D0000CD102E0BEF1000F08D00DF1080E864477
:1076E0009EF8018046EA08088EF8018000F059F8FB
:1076F000E9D1491C0C29DDD37606360E7F1E082FF2
:10770000D6DA02A800900823602200F055F8FEF7B0
:1077100088FF00F04CF801260027002000216FF0C0
:107720000B0202FB0712121992F8922080234FF0ED
:10773000080C03EA020E1DB1BEF1000F0CD102E0ED
:10774000BEF1000F08D00DF1080E86449EF80180AE
:1077500046EA08088EF8018000F023F8E9D1491CB8
:107760000C29DCD37606360E7F1C082FD5DB02A849
:10777000009008236022082100F01FF808E00FF2B3
:107780004C0000901023602200210020FFF7A8FE8B
:107790004FF47A7000F08CF8FEF743FF22B0BDE89A
:1077A000F081401CC0B25B08BCF1010C70477F2126
:1077B0000DF1090002F0FCB80021002090E6000065
:1077C0004C4F474F494E2020424D500000000000D2
:1077D00000000000000000000000000000000000A9
:1077E0000000000080C0E0F0F8FCFEFEFCF8F0E0D5
:1077F000C080C0E0F0F8FCFEFEFEFC783080C0C027
:1078000000189CCEE6F0F8FCFEFEFCF8F0E0C0E0CC
:10781000F0F87C0000000000000000000000000004
:107820000000000000000000000000000000000058
:107830000000000000000000000000000000000048
:107840000000001F0F07030103070F1F3F7F7F3F4B
:107850001F0F07030103070703191C0E6773391C69
:107860000E07030103070F1F3F7F7F3F1F0F070313
:107870000100000000000000000000000000000007
:10788000000000000000000000000000DFF80C16FF
:1078900031F810007047DFF8081688607047DFF88D
:1078A0000006806870472021DFF8F80502F080B8F4
:1078B000142100E00A214843DFF8E41548604868D5
:1078C0000028FCD17047DFF8E0154FF400620A6130
:1078D0004FF480520A61002808680AD120F4404021
:1078E00040F440500860086820F4402040F44030E4
:1078F00009E020F4804040F430400860086820F43B
:10790000802040F430200860704738B502F054F809
:10791000102002F0D5F8DFF88845207820B101204A
:1079200002F0C8F8082502E002F0C4F80025DFF8EC
:107930007C05416841F4D00141F404414160016893
:1079400041F080710160012002F04FF8012002F047
:107950004FF8392002F082F80028FAD0207800B1E0
:10796000022002F048F802F04DF8A842FBD10121B4
:10797000052002F04FF8012140F20D6002F053F8AB
:107980000121032002F058F8207820B10120BDE841
:10799000324002F03CB831BD80B501464FF0006086
:1079A00002F041F94FF4A06002F00CF914208DF8B8
:1079B000000002208DF8010000208DF80200012057
:1079C0008DF8030000A802F002F9122000F004F87C
:1079D000172000F001F801BD8DF8000000208DF89F
:1079E00001008DF8020001208DF8030000A802F0CC
:1079F000EEB83EB50121DFF8B80401F0DCFC202030
:107A0000ADF8000048208DF80300DFF8A84400A975
:107A1000204601F067FC1020ADF80000042000F0C3
:107A200066F80521012001F0EFFC202001900020E4
:107A30008DF808000C208DF8090001208DF80A004F
:107A400001A802F005F91020ADF8000000208DF823
:107A50000300DFF8645400A9284601F043FC4FF40A
:107A60000040ADF8000003208DF80200102000F067
:107A70003EF8402000F041F8082000F02FF80420E4
:107A800000F02CF80320ADF80000482000F02FF89B
:107A90004FF4806000F03DF8082000F02AFA4FF41F
:107AA000807000F036F80120ADF80000102000F0E2
:107AB00033F84FF4006000F038F84FF4805000F0D5
:107AC00034F84FF4005000F030F84FF4804000F0EC
:107AD0002CF84FF4007000F010F837BDADF800003E
:107AE00000208DF8030000A9284601F0FBBB8DF8AB
:107AF000030000A9204601F0F5BBADF8000003200B
:107B00008DF8020010208DF8030000A9284601F02E
:107B1000E9BBADF8000004208DF8030003208DF8C8
:107B2000020000A9284601F0DDBBADF800000320EB
:107B30008DF8020004208DF8030000A9284601F00A
:107B4000D1BBF0B591B04FF42044DC4D284602F093
:107B5000C5F8DB480590D148069000200790022028
:107B600008900020099080200A904FF480700B90BC
:107B70004FF480600C9020200D904FF400500E9038
:107B800000200F9005A9284602F0F5F801212846AB
:107B900002F00CF901220221284602F011F9C94D28
:107BA000284601F047FC00F060F84FF46027029788
:107BB0000020039002208DF8100000A9284601F053
:107BC00062FCC14E304601F035FC00F04EF80297E1
:107BD0000020039001208DF8100000A9304601F02C
:107BE00052FC072302220421284601F0A0FC0723AF
:107BF00001220321284601F09AFC052301220221DB
:107C0000304601F094FC0121284601F063FC01217B
:107C1000284601F056FC0121304601F052FC28466E
:107C200001F06AFC284601F06CFC20B12046441E9D
:107C30000028F7D117E0304601F05EFC304601F035
:107C400060FC0028FAD1304601F05EFC304601F0BD
:107C500060FC0028FAD10121284601F05FFC0121D7
:107C6000304601F05BFC11B0F0BD00200090012017
:107C70008DF804008DF80500704700B585B04FF40D
:107C8000E06001F09FFF86480078002814BF2F2095
:107C90000720ADF8040040F2E730ADF808000020FE
:107CA000ADF80A00ADF8060001A94FF0804002F0DF
:107CB000ABF800F069F802F0FDF8012200F064F87A
:107CC00002F0F0F800F060F802F0E2F81C2000F09A
:107CD0002FF805B000BD1FB54FF4E06001F072FF52
:107CE0006F480078002814BF2F200720ADF804004B
:107CF0003120ADF808004FF48070ADF80A00002084
:107D0000ADF80600714C01A9204602F07DF8012172
:107D1000204602F0CFF801220121204602F0C2F8ED
:107D20000121204602F0B4F81D2000F001F81FBD2B
:107D30008DF8000000208DF8010001208DF8020070
:107D40008DF8030000A801F042BF10B500F01CF848
:107D500002F0BAF800205E4C04EB80014A6812B1D0
:107D60004A68521E4A60401C0828F5DB59480168E1
:107D7000491C01602078411C2170142803D3FEF7B0
:107D8000F3FA0020207010BD01214FF080407047B1
:107D900010B501214D4802F097F8414C606810B1D0
:107DA0006068401E60604C48007830B10020FFF7EA
:107DB0006DFDFEF757FB49490860A0686178484AA5
:107DC00048B1A068401EA060002919BF4020506043
:107DD00040201060C943A06810B9402050600021C5
:107DE000617010BD38B5384C45F64D034FF4584519
:107DF000694391FBF3F292B2684390FBF3F189B2CD
:107E0000204601F0DCFB0221204601F0DBFB354976
:107E1000204601F0CEFB01224FF4A0712046BDE8C0
:107E2000384001F060BB38B5274C4FF4A0712046B4
:107E300001F0DAFB78B1A56A204601F0B7FB854274
:107E400002D31748002181604FF4A0712046BDE89D
:107E5000344001F0D6BB31BD10B582B0164C58B1DC
:107E60000821144801F0A5FA4FF4806100F03EF8B3
:107E700000F03AF801210BE04FF4806000F039F88F
:107E80004FF4807000F035F800F02EF84FF4806168
:107E900000F02CF86420FFF70BFD13BD1C3200200E
:107EA00088080020A0310020040801400010024092
:107EB00000023000000C01400008014008000240B0
:107EC0004C240140002401400028014000040040EF
:107ED0009C31002020320020E4310020E8310020D5
:107EE00010080140000280004FF48071204601F02C
:107EF00060BAADF8000010208DF8030003208DF863
:107F0000020000A9204601F0EDB90000002201F0B6
:107F1000F3BF000062B38B0708D0521E11F8013B7B
:107F200000F8013B00F024808B07F6D1830740F076
:107F3000208000BF103A07D330B4B1E83810103AAF
:107F4000A0E83810F9D230BC530724BFB1E80810BC
:107F5000A0E8081044BF51F8043B40F8043BD207A6
:107F600024BF31F8022B20F8022B44BF0B7803709A
:107F70007047083A07D3B1E80810083A40F8043BC4
:107F800040F804CBF7D25307E4E70000704710B580
:107F90004FF41852DFF8D81BDFF8D80BFFF7CAFFF1
:107FA000DFF8D40B002100220B460C461EC010BD8A
:107FB00010B5002208E0135CA3F16104E4B21A2CAE
:107FC0003CBF203B1354521C8A42F4DB10BD2DE908
:107FD000FF4180460E46DFF89C4B04F20047102517
:107FE0000B22394601A8FFF795FF0B2101A8FFF7E7
:107FF000DFFF0B22414601A801F098FF98B907F175
:108000001C00017831704178717007F11A0000A9E5
:1080100002780A7042784A70BDF8000004EB4020F4
:1080200000F5007003E020376D1ED9D1002004B0A8
:10803000BDE8F08120281CBF0D280A2801D10120AD
:1080400070470020704710B5044600E0641C20789B
:10805000FFF7F0FF0028F9D114F8011B0A462D297B
:1080600006D02B2906D103E00A2303FB0010303889
:1080700014F8011BA1F13003DBB20A2BF4D32D2A33
:1080800008BF404210BD2DE9F04180460D463D211C
:1080900008F1D80001F07CFF002811D000F091F821
:1080A00080B2002818BF012814D10746A862002416
:1080B0000A263D21242000FB048001F069FF0028EE
:1080C00079D000F07EF880B22FB9A0F16401B1F54B
:1080D000967F05D96FE0A0F1D401B1F5077F6AD88A
:1080E0007043002C0CBF28616861641C022CE0DB2B
:1080F0003D2108F1480001F04BFF00285BD000F063
:1081000060F880B2A0F13C01B1F56B7F53D26421DD
:108110004843E8613D2108F16C0001F039FF002877
:1081200049D000F04EF880B2A0F11001092942D2E6
:1081300028623D2108F1900001F02AFF00283AD082
:1081400000F03FF880B2411E192934D27043A86173
:108150003D2108F1B40001F01BFF60B300F031F8DD
:1081600080B2A0F16401332925D2E8623D2108F1F3
:10817000FC0001F00DFFF0B100F023F880B2002800
:1081800018BF012817D168623D2108F5907001F0F1
:10819000FFFE80B100F015F880B228633D2108F59C
:1081A000A27001F0F5FE30B100F00BF880B20028AB
:1081B00018BF012801D0002001E068630120BDE85C
:1081C000F081401C3FE72DE9F047F2B004468846B5
:1081D00000264FF4B47118A8FFF798FEDFF89C79D9
:1081E00000F074FB4FF0240900AC0025252100A805
:1081F000FFF78CFEB6F5007F3EDAF05D2855761C61
:108200000A2818BF0D286AD10020285500A8FFF7BA
:108210000FF880B268B300A94018A0F1010A01E08C
:10822000AAF1010A00A8824505D39AF80000FFF7D9
:1082300001FF0028F4D100208AF8010000AD00E021
:108240006D1C287818B1FFF7F5FE0028F8D100A8BA
:10825000A8420ED0AAEB0500801C80B200A9002223
:1082600004E015F8013B01F8013B521C92B2824236
:10827000F7D39DF8000048B9B6F5007FB5DB0020C4
:1082800018A909FB0011097869BB34E0002507EB48
:108290008500D0F800A25046FEF7CAFF00A911F8E9
:1082A000012BA2F141031A2B38BF20321AF8013BEF
:1082B000A3F1410CBCF11A0F38BF2033401E80B22D
:1082C00030B19A42EBD003D06D1C0A2DD4DADEE730
:1082D00000A918A809FB050001F066FECCE76D1C9B
:1082E000242D87DBC8E7401C0A28C9DB0AA918A887
:1082F000FFF7C9FE08B901264FE00026DFF88078B5
:1083000028220EA907F11000FFF704FE0A2438699D
:1083100090FBF4F20FF6900118A8FFF710F87869B7
:1083200090FBF4F20FF68C0121A8FFF708F8F8692A
:1083300000F065F92AA8FFF702F83A6A0FF68C01F7
:1083400033A8FEF7FCFFB869B0FBF4F20FF6880122
:108350003CA8FEF7F4FFFA6A0FF6880145A8FEF77D
:10836000EEFFBA6A0FF688014EA8FEF7E8FF7A6AB8
:108370000FF6840157A8FEF7E2FF3A6B0FF6800173
:1083800060A8FEF7DCFF7A6B0FF6800169A8FEF7A4
:10839000D6FF386BDFF8EC1708604FF49671404653
:1083A00001F006FBDFF8D07776B1002407EB8405F7
:1083B000E96B404601F01AFE6969404601F016FE7D
:1083C000641C0A2CF2DB0FE0002418A809FB04014E
:1083D000404601F00BFE07EB84004169404601F086
:1083E00005FE641C0A2CF0DB304672B0BDE8F08755
:1083F0002DE9F043D5B00020ADF800004FF49671A0
:108400000AA8FFF783FD0A24DFF87457286990FB58
:10841000F4F20FF2947100F0F8F800F0ECF8DFF8E5
:108420005867716900F0E8F8686990FBF4F20FF2A0
:10843000847100F0EAF800F0DEF8B16900F0DCF8D1
:10844000E86900F0DCF800F0E0F800F0D4F8F16939
:1084500000F0D2F82A6A0FF2747100F0D6F800F03A
:10846000CAF8316A00F0C8F8A869B0FBF4F20FF25C
:10847000687100F0CAF800F0BEF8716A00F0BCF84C
:10848000EA6A0FF2607100F0C0F800F0B4F8B16A67
:1084900000F0B2F8AA6A0FF2587100F0B6F800F0D6
:1084A000AAF8F16A00F0A8F86A6A0FF24C7100F0BD
:1084B000ACF800F0A0F8316B00F09EF82A6B0FF2D8
:1084C000407100F0A2F800F096F8716B00F094F89B
:1084D0006A6B0FF2387100F098F800F08CF8B16B0D
:1084E00000F08AF80FF2307800F045F94046FFF7C7
:1084F0006EFD00F03AF918D00AA8FEF799FE024680
:10850000BDF8000004EB401080F81C24110A00F0B4
:1085100067F881550AA8FEF78BFE02460AA938467D
:10852000FFF7F8FC00F011FA4BE00FF2F86900F0E9
:1085300022F94846FFF74BFD010004F21646DFF82A
:10854000487616D0FE220AA8FFF7E4FC00F008F9EE
:1085500004F58460B9E80E000EC0FE220AA904F5F5
:108560000060FFF7E7FC00207075376200F0F1F85B
:1085700001E000F0F5F8B8E8070007C50FF6BC0504
:10858000062229462046FFF7D5FC0622294604F597
:108590000070FFF7CFFC0AA8FEF74AFE05462A4600
:1085A0000AA904F5C060FFF7C5FC002084F80B049D
:1085B000C4F8167402203071B571280AF07100F009
:1085C000EDF942F60C0001190022CA760A774A76C4
:1085D0000251002088600861C86055B0BDE8F08392
:1085E00080F81D14781B00F50070411200EB9150CB
:1085F00080120121704701A90AA801F0F7BC64218B
:10860000B0FBF1F20FF2B851704701A8FEF797BE28
:108610002DE9F04FCDB00020ADF800000FF2F85674
:1086200000F0A9F83046FFF7D2FC00F09EF8DFF822
:1086300048951ED001A9FFF7C6FD00287AD001A8F1
:10864000FEF7F6FD0646BDF8000004EB401080F88A
:108650001C64310AFFF7C4FF00F8091001A8FEF7F7
:10866000E7FD024601A93846FFF754FC00F06DF91A
:1086700060E00FF2B05A00F07EF85046FFF7A7FC1A
:10868000010004F21647DFF8008517D0FE2201A88A
:10869000FFF740FC00F064F804F58460BAE80E00CF
:1086A0000EC0FE2201A904F50060FFF743FC002084
:1086B0007875C7F8208000F04CF801E000F050F821
:1086C00007CE07C50FF27476062231462046FFF723
:1086D00031FC0622314604F50070FFF72BFC002622
:1086E000002509EB850ADAF83CB05846FEF7A0FDF4
:1086F00000F045F8DAF83C00FEF79AFD8619DAF842
:1087000014B05846FEF794FD00F039F8DAF814007A
:10871000FEF78EFD86196D1C0A2DE2D3002084F829
:108720000B04C4F8168402203871BE71300AF87147
:1087300000F034F942F60C0001190022CA760A77DB
:108740004A760251002088600861C8604DB0BDE8DB
:10875000F08F032084F83A04FE2084F83C0470472C
:108760004FF418512046FFF7D1BB0700DFF804444F
:1087700004F20045704700AA0DF10201704702465D
:108780005946301900F5C060FFF7C4BB2DE9F0472A
:10879000D0B004468846DFF8DC93B8F5805F0BD193
:1087A0004FF40072494601F0C1FB00280FD04FF48E
:1087B0000072214648460FE0B8F5205F0FD109F559
:1087C00000754FF40072294601F0B0FB002878D004
:1087D0004FF4007221462846FFF79CFB71E009F236
:1087E0000047DFF89453B8F5804F2BD14FF4007257
:1087F000394601F09BFB002863D000F067F80120A8
:10880000687010260FF210470C22214600A8FFF7CF
:1088100081FB0B22394600A801F088FB40B9A07EFD
:10882000688201202874207F40B10120287048E030
:108830002034761EE8D1287C0028F6D00020287449
:1088400028803EE0A8F5004ABAF5005F39D808EB69
:108850000900A0F5F4464FF400723146204601F0BD
:1088600065FB28B14FF4007221463046FFF752FBFA
:108870004FEA5A20801C698A88421CD105A93046DB
:10888000FFF7A1FCF8B905A8FEF7D2FC698A09EB4D
:10889000411181F8DC03000A81F8DD03F01BFFF7CA
:1088A000A2FE415505A8FEF7C3FC024605A93046C5
:1088B000FFF730FB05E0A8F5FC4005EB9020012117
:1088C000417000F042F850B0BDE8F0874FF40072FC
:1088D00021463846FFF71EBB38B504460D46FFF764
:1088E00055FB25B94FF400720FF2503121E0A14938
:1088F000B5F5805F08BF4FF400721AD0B5F5205F60
:1089000004D14FF4007201F5007112E0B5F5804F0B
:1089100004D14FF4007201F580610AE0A5F5004032
:10892000B0F5005F0AD84FF4007205F1006101F55F
:108930008C412046BDE83840FFF7ECBA4FF4007197
:108940002046BDE8344001F033B8F8B501F0C2F874
:1089500000208949425CD2B1002242548402844DF5
:10896000281901F062FB83482618002736F8021BFD
:108970003819281801F048FB042803D001F0B4F896
:108980000420F2BDBF1CB7F5806FEFD302E0401C9E
:108990001028DFD301F0A8F80020F2BD70B5754CA7
:1089A00001F098F80025724E06EB852001F03DFBA2
:1089B0006D1C092DF8DB002534F8021B701901F03D
:1089C00023FB042801D0042070BDAD1CB5F5185F51
:1089D000F2DB01F089F8002070BD2DE9F04142F68C
:1089E0001804644D6619694F327A2AB9400238601A
:1089F0004802786001203072307A012831D1605904
:108A000078B905F5185839684046FFF765FF4022E8
:108A10009821404601F01EFB4FF4E0706051402069
:108A20000CE040229821B868401900F5185001F078
:108A300011FB605940386051B8684030B86040213F
:108A4000012001F0B2FB3021012001F038FB386831
:108A5000403038607868403878604D4881684039E7
:108A60008160786838B96051B8603860494803213E
:108A7000017000203072BDE8F0812DE9F04142F62E
:108A80001C043C4D625940326619434F33792BB96F
:108A90004002386048027860012030713079012846
:108AA0002FD100203D490AE05B1903F5185310F857
:108AB00001C083F800C0401C63595B1C63516359BB
:108AC0009342F1D3DFF8D880B8F800003968411834
:108AD00039607A68101A7860C00507D100206051AB
:108AE000A1F5007105F51850FFF750FE2848816880
:108AF000B8F80020891A81604FF44051022001F03B
:108B0000EFFA786800281EBF22480078042806D1B2
:108B100000206051012101F0AFFC00203071BDE860
:108B2000F08110B5FDF7F4FDFEF782FDFEF752FD72
:108B3000FEF77EFD1B4C01202070FFF728FAFFF79F
:108B400057FC00202070FDF76CFD00220FF2E001C1
:108B50000020FCF717F94FF47A70FEF7A9FEFDF735
:108B600060FD4FF47A70BDE81040FEF7A1BE000032
:108B700000C00008CC080020B00600200000002043
:108B80007006002030080020188DDD40D031002014
:108B9000C031002068310020DC3100200831002085
:108BA0006A3100202808002053746254656D703DBE
:108BB00025640000576B54656D703D25640000000E
:108BC000536C7054696D653D256400005261746595
:108BD000645F503D2564000054656D705374703DB2
:108BE000256400004F6666566F6C743D2564000076
:108BF00054656D703D25640048616E643D256400D8
:108C00005A65726F505F41643D256400506F727405
:108C100061626C653D256400434F4E464947202004
:108C2000545854004C4F474F494E2020424D50005D
:108C3000436F6D706C657465642E0000EB3C904D65
:108C400053444F53352E30000201080002000250F9
:108C500000F80C000100010000000000000000000E
:108C6000000029A298E46C4E4F204E414D45202033
:108C70002020464154313220202033C98ED1BCF00F
:108C80007B8ED9B800208EC0FCBD007C384E247D80
:108C9000248BC199E83C01721C83EB3A66A11C7CD1
:108CA00026663B07268A57FC750680CA028856024C
:108CB00080C31073EB33C98A461098F766160346D3
:108CC0001C13561E03460E13D18B7611608946FC89
:108CD0008956FEB82000F7E68B5E0B03C348F7F316
:108CE0000146FC114EFE61BF0000E8E60072392625
:108CF000382D741760B10BBEA17DF3A66174324E9E
:108D0000740983C7203BFB72E6EBDCA0FB7DB47DDE
:108D10008BF0AC9840740C487413B40EBB0700CDB4
:108D200010EBEFA0FD7DEBE6A0FC7DEBE1CD16CDD9
:108D300019268B551A52B001BB0000E83B0072E8BF
:108D40005B8A5624BE0B7C8BFCC746F03D7DC74634
:108D5000F4297D8CD9894EF2894EF6C606967DCBD4
:108D6000EA030000200FB6C8668B46F86603461C6F
:108D7000668BD066C1EA10EB5E0FB6C84A4A8A46D7
:108D80000D32E4F7E20346FC1356FEEB4A5250065E
:108D9000536A016A10918B4618969233D2F7F69176
:108DA000F7F64287CAF7761A8AF28AE8C0CC020A36
:108DB000CCB80102807E020E7504B4428BF48A5650
:108DC00024CD136161720B40750142035E0B49753E
:108DD00006F8C341BB000060666A00EBB04E544C1D
:108DE00044522020202020200D0A52656D6F7665A8
:108DF000206469736B73206F72206F7468657220D2
:108E00006D656469612EFF0D0A4469736B2065729C
:108E1000726F72FF0D0A507265737320616E792054
:108E20006B657920746F20726573746172740D0ABA
:108E300000000000000000ACCBD855AAF8FFFFFFEF
:108E4000FFFF000009490860704709490860704742
:108E500008490860704705484AF6AA210160704732
:108E600002484CF6CC4101607047000000300040E1
:108E700004300040083000404FF4001C1CEB410F50
:108E800094BF1CEB430F09E041EA030C50EA4C0C81
:108E900052EA0C0C03D28B4208BF8242704714BFC7
:108EA000994290427047000070B44FF0004591EA3B
:108EB000030C44BF6B4000F047B900BF841A71EB4C
:108EC000030603D2001BB141121973414FF4001C79
:108ED0001CEB410F34BF7CEB430443E00C0DA4EBCF
:108EE0001356352E50DC45EAC323DB0A45EAC1217F
:108EF000C912B6F120050DDD63FA05F6EB4086EAEE
:108F00000305124218BF45F00105C01851F10001D8
:108F10000CD213E062FA06F5F2405540F3415A4094
:108F2000B340F3405A408018594107D349085FEADB
:108F300030005FEA350528BF45F0010501F58011D5
:108F4000420875F1004250F1000041EB045170BC41
:108F50004FF4001C1CEB410F38BF70470020090D77
:108F6000090570471CEB410F10D252EA43060BD0A3
:108F7000BCEB410F05D80C0DAB43661E342EB5DD9E
:108F800002E0AB438018594170BC704770BC704719
:108F9000B0B581EA030C0CF0004C40F2FF7515EA05
:108FA00011541DBF15EA1357AC42AF4239E0E41922
:108FB00023EA455343F48013C90241F0004141EADA
:108FC000505EC7021100A7FB020200284FF000000C
:108FD000EEFB01204FF00001E3FB072118BF42F038
:108FE0000102401800214941E3FB0E01A4F5806411
:108FF0000F0302D252004041494154F101046CDD9B
:10900000470872F1004250F1000051EB0451A1F504
:1090100080115CBF41EA0C01B0BD4CEA0551002053
:10902000B0BD05EA1357AC4214BFAF4241E050EA6D
:10903000410E1CBF52EA430E02E061460020B0BD63
:1090400024423C441BD15FEA070EF6D0090302BF5D
:1090500001460020AEF1140EB1FA81F7AEEB070421
:1090600001FA07FE0C37C7F1200100FA07F7C840E4
:109070004EEA000E23EA455343F48013A2E733F08F
:109080000043B3FA83F704BFB2FA82FE77440B3F82
:10909000E41BB7F1200E2FBF02FA0EF3BB40C7F15D
:1090A000200E22FA0EFE38BF43EA0E03BA40641CBB
:1090B00082E750EA410E14BF52EA430E6FF00001FE
:1090C0004FF4001717EB430F8ABF194617EB410FF8
:1090D000B5E74CEA05510020B0BDD4F10104B4F16C
:1090E00020070FDAC4F12007520828BF42F001021E
:1090F00010FA07F501FA07F7E1BF2A43E0403843C9
:10910000E1400FE0352C98DCC7F1200452EA400220
:1091100020FA07F218BF42F0010231FA07F0A1402D
:109120000A43002172F1004250F1000051EB0C01A2
:10913000B0BD000070B44FF0004591EA030F44BF8A
:109140006B40FFF7BBBE00BF841A71EB030604D26D
:109150006E40001BB141121973414FF4001C1CEB0F
:10916000410F34BF7CEB430684E00C0DA4EB135697
:10917000362E7DDC012E43DC45EAC32343EA5253FD
:1091800012BFD20292025B08240545EAC12141EADE
:109190005051D2EBC020994125D407D1B0FA80F6C6
:1091A00010FA06F164D00020203608E0B1FA81F60A
:1091B000B140C6F1200220FA02F21143B0404FEA5A
:1091C000F474B4EB465434F001064FEA74040AD840
:1091D000D6F50016760D04F00044F04061FA06F270
:1091E0005040F1404840C00A40EA415021F000415F
:1091F00028BF5FEA500550F1000044EBD12137E071
:1092000045EAC323DB0A45EAC121C90AB6F12005B4
:109210000EDD42EA0242120CC5F1200603FA06F600
:10922000EB4042EA06056D42984161F100010DE014
:1092300062FA06F5F240554063FA06FC82EA0C0237
:10924000F3405A406D42904161EB030111F4801FDD
:1092500005D1641E620502D06D004041494121F4F0
:109260008011430875F1004350F1000041EB0451B7
:1092700070BC70471CEB410F15D223F0004352EA3B
:1092800043060BD04FEA4C0CBCEB410F04D80C0D3D
:10929000661E342EB7DDEBE7801A994150EA41068D
:1092A00008BF0021E4E708BF1CEB430F28BF6FF0A5
:1092B0000001DDE74FF4001C1CEB410F94BF1CEBD9
:1092C000430F09E041EA030C50EA4C0C52EA0C0C43
:1092D00003D2994208BF9042704714BF8B4282422A
:1092E000704700002DE9F0410022CC7804F00F0314
:1092F000E40644BF8C7823430C8801250F26E7B28F
:1093000017B3D0F800C005FA02F7BE460EEA04080B
:10931000F04514D14FEA820E06FA0EF82CEA080C3A
:1093200003FA0EFE4EEA0C0C91F803E0BEF1280F92
:1093300008BF476103D0BEF1480F08BF0761521C48
:10934000082AE0D3C0F800C0B4F5807F26D3D0F857
:1093500004C0002202F1080705FA07F7BE460EEA2C
:109360000408F04515D14FEA820E06FA0EF82CEAF1
:10937000080C03FA0EFE4EEA0C0C91F803E0BEF165
:10938000280F08BF476191F803E0BEF1480F08BFFE
:109390000761521C082ADDD3C0F804C0BDE8F08183
:1093A00000228068084218BF012210467047016100
:1093B00070474161704770B51C4A00284CBF9469E2
:1093C0001468C0F3034583B2460D3601B34000F480
:1093D0004016B6F5401F06D124F07064156825F0DC
:1093E0007065156008E0C60243BF032606FA05F55E
:1093F000AC439C4344F0706401B11C43002801D588
:10940000946170BD146070BD30B501F0030292002C
:1094100021F00301064BCC580F259540AC43CC50AE
:10942000CC5890402043C85030BD0000040001409B
:109430000800014080B56649884208D101214FF4F7
:10944000007000F002FB00214FF4007016E061494B
:10945000884208D101214FF4806000F0F6FA002123
:109460004FF480600AE05C4988420BD101214FF43F
:10947000004000F0EAFA00214FF40040BDE804404B
:1094800000F0E3BA01BD4268544B1A400B681A431E
:109490000B7942EA032242608268514B1A40CB6842
:1094A0001A438B681A434B7942EA43028260C26ACC
:1094B00022F47002097C491EC9B242EA0151C1621C
:1094C00070470029816812BF41F001014908490035
:1094D000816070470029816814BF41F4807121F4D4
:1094E000807181607047C9B2002A426814BF11437D
:1094F00022EA010141607047816841F00801816002
:1095000070478068C00806E0816841F0040181600E
:1095100070478068800800F001007047002981686A
:1095200014BF41F4A00121F4A0018160704770B51F
:1095300007240A290BD3A1F10A0505EB4505C668E6
:10954000AC4026EA0404AB402343C36008E001EBCF
:1095500041050669AC4026EA0404AB40234303619D
:109560001F23072A0AD2521E02EB8202446B934049
:1095700024EA030391401943416370BD0D2A0AD2C6
:10958000D21F02EB8202046B934024EA0303914052
:109590001943016370BD0D3A02EB8202C46A934025
:1095A00024EA030391401943C16270BDC06C80B2CC
:1095B000704742680B4B1A4011434160704741624B
:1095C000826270474268520951EA42114160704715
:1095D0000024014000280140003C0140FFFEF0FF54
:1095E000FDF7F1FFFFFD3FFF10B500224368CCB24D
:1095F0002340006810EA112F1CBF002B01221046E7
:1096000010BD090AC943016070470000010000BF96
:1096100009D0B0FA80F18840C91CC1F58461090500
:1096200001EBD02140057047F446400D40EAC120CF
:10963000490006D200F00EF8004248BF6FF000402B
:10964000604700F007F84FF0004188428CBF0846A1
:109650004042604740F00040490DA1F58061491C3F
:1096600005D4D1F11F0154BFC840C01770474FF057
:10967000000070473E480088704738B53C4C3D4D6F
:10968000287848B101202080FCF7D0FF60600020DE
:109690002870312000F01AF86068FCF7CBFF97289B
:1096A00024BF0020208031BD38B504460D4600F0AF
:1096B0008AF8322000F0C0F8204600F0BDF82846B5
:1096C00000F0BAF8BDE8314000F0A0B800B585B0B0
:1096D0008DF800002849097B0029034614BF192290
:1096E0001D22012100A800F03CF99DF8000005B002
:1096F00000BD80B52048007BD0B100212120FFF7BC
:10970000D3FF40212220FFF7CFFF00212320FFF7C6
:10971000CBFF7F213020FFF7C7FF2A213220FFF740
:10972000C3FF03213320FFF7BFFF3721202011E0C3
:1097300000212A20FFF7B8FF02210E20FFF7B4FF17
:1097400003212A20FFF7B0FF00212B20FFF7ACFFF9
:1097500001212A20BDE80440A6E780B50F20FFF7CD
:10976000B5FF33280CBF012000200349087301BD59
:10977000FC3100203C32002074080020002800E06A
:10978000401EFDD1704780B5FDF714FFC020ADF835
:10979000000003208DF802001C208DF8030000F06B
:1097A00001F801BD00A95848FFF79CBD564A0129A0
:1097B00003D101461046FFF7FABD19B9014610461C
:1097C000FFF7F7BD704780B50121082000F02BF9A5
:1097D000C020ADF8000014208DF8030003208DF8A0
:1097E0000200FFF7DFFF00F00EF800F057F800F07E
:1097F00058F800F051F8002100F051F800F04CF852
:1098000000F001F801BD00214020CFE780B5FFF74F
:10981000FAFF002100F043F800F03EF800F041F8B4
:1098200000F03AF800F03AF800F036F8FFF7EBFFF6
:109830000220BDE80240A1E738B50446082508E04B
:1098400000F02DF800F028F800F02BF800F024F8D4
:1098500064002846451EC0B230B1FFF7D4FF200691
:109860004CBF01210021EBE7FFF7CDFF00F016F818
:10987000FF2400F011F800F043F848B900F011F8A7
:1098800000F00AF8FFF7BFFF00F006F8012032BD34
:10989000641EEED1002032BD02206FE7012180203E
:1098A00084E70121402081E770B5044608250026A1
:1098B000FFF7F4FF0DE0FFF7A6FFFFF7EDFFFFF75F
:1098C000F0FFFFF7E9FF760000F01AF808B146F064
:1098D00001062846451EC0B20028ECD1FFF793FFD1
:1098E000002C0CBF01210021FFF7D9FFFFF7D4FFA7
:1098F000FFF7D7FFFFF7D0FFFFF785FFF0B270BD8E
:1099000080210148FFF74CBD000C0140F8B504462A
:109910000D461646002703B14027FFF754FF70009D
:10992000C0B2FFF789FF384601E014F8010BFFF7DA
:1099300083FF2846451EC0B20028F6D134E038B572
:1099400004460D46FFF73FFF6800C0B2FFF774FF03
:109950000020FFF771FF2046FFF76EFFBDE83140A2
:1099600054E7F8B504460D4616461F46FFF72BFF91
:109970007600F0B2FFF760FF3846FFF75DFFFFF7B4
:1099800022FF46F00100C0B2FFF756FF03E0FFF7E9
:109990008BFF04F8010B2846451E28B1EDB2002DBF
:1099A0000CBF00200120F2E7BDE8F1402EE70000E7
:1099B0000022FDF76DBC00003348016841F0010151
:1099C00001604168314A114041600168304A1140EC
:1099D0000160016821F480210160416821F4FE01E9
:1099E00041604FF41F01816070472A490860704749
:1099F0002A490860704728490A68920850EA82009C
:109A0000086070472448006800F00C007047244943
:109A100008607047234A0029116814BF084321EAEF
:109A2000000010607047204A0029116814BF0843E5
:109A300021EA0000106070471C4A0029116814BF19
:109A4000084321EA000010607047194A0029116894
:109A500014BF084321EA000010607047002142094A
:109A6000094B012A08BF1A6803D0022A0CBF1A6AE0
:109A70005A6A012300F01F0003FA00F0024218BFE7
:109A80000121084670470000001002400000FFF866
:109A9000FFFFF6FE00004242041002406000424216
:109AA000D800424214100240181002401C1002401C
:109AB0000C100240DFF8D4100A6802F0380206E009
:109AC000DFF8C8100A6822F010020A600A68104322
:109AD00008607047FFE7DFF8B800DFF8B8100160F2
:109AE000DFF8B41001607047FFE7DFF8B0000168ED
:109AF00041F080010160704738B5054600F015F867
:109B000004280DD1DFF89440206840F00200206066
:109B1000656000F006F8216841F6FD721140216091
:109B200032BD206840F0400020604FF4302039E022
:109B300070B504460D4600F011F804280CD1174EFC
:109B4000306840F001003060258000F007F831688F
:109B500041F6FE721140316070BD08804FF4005034
:109B600020E00F490860704704200D490A68D207B9
:109B700001D5012070470A68520701D502207047BD
:109B80000968C90648BF0320704700000020024052
:109B90000420024023016745AB89EFCD102002402D
:109BA0000C20024010B5FFE70446FFF7DDFF03E09D
:109BB0002CB1FFF7D9FF641E0128F9D004B90520A4
:109BC00010BD00001B4908431B490860704770B571
:109BD00003781A460121C478ECB1174B1B6803F4D3
:109BE000E063C3F5E0631B0A4478C3F10405AC40AD
:109BF00085780F2626FA03F32B4023431B010F4CD5
:109C00001355007842110E4B00F01F0001FA00F0CE
:109C100043F8220070BD50110A4A03F01F03994017
:109C200042F8201070BD084A1140084307490860F7
:109C3000704700000000FA050CED00E000E400E0D1
:109C400000E100E080E100E080FFFF1F08ED00E0A0
:109C500030B50168CB431F4982792AB30A4614689C
:109C60002340136053680468A34353600379CC18FE
:109C7000236805682B43236093680468A3439360BB
:109C8000D3680468A343D36043790568102B07D1D8
:109C9000916829439160D16800680843D06030BD65
:109CA000CC182068284303E000790C18206818407D
:109CB000206030BD0021074A136803405269024208
:109CC0001CBF002B01210846704700BF02490860F5
:109CD00070470000000401401404014001684FF681
:109CE000FE72114001600021016041608160C1602D
:109CF0003749384A90421DD0374A904221D0374ADE
:109D0000904225D0364A904229D0364A90422DD0F2
:109D1000354A904203D1086840F4700029E0334A84
:109D2000904203D1086840F0706022E03049314A27
:109D3000904203D1086840F00F001AE02E4A90428A
:109D400003D1086840F0F00013E02C4A904203D1A0
:109D5000086840F470600CE0294A904203D108681A
:109D600040F4704005E0274A904203D1086840F46F
:109D700070200860704702686FF30E128B681A43F8
:109D80000B6A1A430B691A434B691A438B691A43CE
:109D9000CB691A434B6A1A438B6A1A430260CA683A
:109DA00042600A6882604968C160704700290168A2
:109DB00012BF41F001014FF6FE7211400160704781
:109DC000002A026814BF114322EA010101607047B2
:109DD00004000240080002401C0002403000024023
:109DE00044000240580002406C00024080000240E3
:109DF00004040240080402401C04024030040240F3
:109E0000440402405804024030B50488DFF8D820EA
:109E1000DFF8BC30984218BF90420ED0B0F1804FAE
:109E20001CBFDFF8B050A84207D0DFF8AC50A84202
:109E30001CBFDFF8A850A84204D14FF68F752C4004
:109E40004D882C43DFF89850A8421CBFDFF894508F
:109E5000A84204D04FF6FF452C40CD882C43048007
:109E60008C8884850C880485984218BF90420AD05B
:109E7000DFF8782090421FBFDFF874209042DFF8AF
:109E80007420904201D1097A01860121818230BD7E
:109E90000029018812BF41F001014FF6FE72114006
:109EA00001807047002A828914BF114322EA010110
:109EB000818170470029018812BF41F080014FF66F
:109EC0007F7211400180704700BFC9430182704713
:109ED000002C01400004004000080040000C00403D
:109EE00000100040001400400034014000400140D8
:109EF000004401400048014000B500BF13009646F1
:109F00009446103928BFA0E80C50FAD85FEA417C8B
:109F100028BF0CC048BF40F8042BC90728BF20F851
:109F2000022B48BF00F8012B00BD000003000020F9
:109F300013F0030F09D0521E22BF13F8010B11F8C2
:109F400001CBB0EB0C00F3D07047121F22BF53F8C7
:109F5000040B51F804CB6045F7D0121D0AD200BAA9
:109F60009CFA8CFCB0EB0C0038BF6FF0000088BF8F
:109F700001207047521E22BF13F8010B11F801CBCC
:109F8000B0EB0C00F6D0521C08BF10467047000022
:109F90000278C9B28A421AB11CBF10F8012FF9E742
:109FA00018BF0020704700005FEA000C830706D04E
:109FB00011F8013B00F8013BB3B18307F8D10A68FF
:109FC000B2F1013323EA020313F0803F02BF40F8ED
:109FD000042B51F8042FF3E711F8013B00F8013B83
:109FE00013B111F8013BF9E760467047024600E003
:109FF000521C1378002BFBD111F8013B137012F89F
:10A00000013B002BF8D1704738B504460D46104887
:10A01000FFF7C8FD05281CBF3420FFF7A2FD294625
:10A020002046BDE83440FFF783BD10B50446A005C7
:10A030000CD10748FFF7B6FD05281CBF3420FFF7F9
:10A0400090FD2046BDE81040FFF756BD10BD000052
:10A05000A086010010B5490001F1804101F5C04121
:10A06000521C521009E010F8013B10F8014B43EA72
:10A07000042321F8023B891C521EF4D110BD490073
:10A0800001F1804101F5C041521C521004E051F829
:10A09000043B20F8023B521EF9D170474FF6F8718D
:10A0A0000840DFF890110860704710B5DFF888218C
:10A0B00052F8203048F68F142340194324E010B59D
:10A0C000DFF8742152F8203048F6BF742340CC06E4
:10A0D00048BF83F01003890648BF83F020030FE0D8
:10A0E00010B5DFF8542152F820304BF68F7423401E
:10A0F000CC0448BF83F48053890448BF83F40053E1
:10A1000043F4004141F0800142F8201010BDDFF817
:10A11000281151F820204BF68F731A4082F44052D8
:10A1200042F4004209E0DFF8101151F8202048F60F
:10A130008F631A4042F40042FFE742F0800241F888
:10A1400020207047DFF8F01051F8202052040AD583
:10A1500051F8202048F68F731A4042F4404242F0F2
:10A16000800241F820207047334951F820205206E0
:10A170000AD551F8202048F68F731A4042F4004265
:10A1800042F0C00241F82020704738E0294A1268A6
:10A1900092B202EBC000294A37E03BE0254909684A
:10A1A00089B201EBC00025493AE0224A126892B216
:10A1B00002EBC000224A2AE01E4A126892B202EB69
:10A1C000C000204A02EB40003F2909D34A091F235F
:10A1D000194208BF521E1204910941F4004105E0E2
:10A1E0004A08C90748BF521C120491090160704710
:10A1F0001049096889B201EBC000124914E00D4A08
:10A20000126892B202EBC0000F4A4908490042F8B6
:10A21000101070470749096889B201EBC0000A496C
:10A2200051F8100080B2704751F810008005800D81
:10A2300070470000505C0040005C00400860004037
:10A24000046000400C600040006000400106090C02
:10A2500041EA10207047000080B5964890F8201021
:10A26000022909D018D3042902D00ED3052913D10D
:10A27000002180F820100CE0C17B28290CD1816AD4
:10A28000406ABDE8044000F07CB90121002000F0E4
:10A29000F3F84FF440512BE101BD38B5854CE57B17
:10A2A0000220FFF7A5FF60840246D8218248FFF70D
:10A2B000E6FE94F8200010B1012803D00AE0BDE8C2
:10A2C000314013E02A2D06D1A16A606ABDE834400E
:10A2D00000F081B9022000F0F9F82421052000F0F7
:10A2E0004BF900210220BDE83440C5E010B5714CA7
:10A2F000628C1AB170492046FDF71CFE6F486168F8
:10A300004160A1688160608C1F2806D0022000F0A7
:10A31000DDF8002020601A218DE0E27B282A18BF9A
:10A320002A2A0FD1607CA17C090441EA0060E17C0B
:10A3300040EA0120217D08436062A07DE17D41EA81
:10A340000020A06220685E49884270D15D480068A4
:10A35000617B884204D3A07B401EC0B2102804D386
:10A36000022000F0B3F8242165E0606AA16A002AA7
:10A3700049D0032A2BD0082A18BF0A2A53D0122A00
:10A3800029D0152A4FD01A2A2DD01B2A27D01D2AB2
:10A3900049D01E2A23D0232A2DD0252A2FD0282A7F
:10A3A00035D02A2A37D02F2A39D0552A3BD05A2ADD
:10A3B0001DD0882A18BF8A2A35D08F2A18BF9E2A16
:10A3C00031D0A82A1CBFAA2AAF2A2CD02FE0BDE882
:10A3D000104000F0C9B8BDE8104000F08FB8BDE8EB
:10A3E000104000F0CDB8BDE8104000F0B5B8BDE8B1
:10A3F000104000F0B5B8BDE8104000F08EB8BDE8E0
:10A40000104000F099B8BDE8104000F023B9BDE855
:10A41000104000F0B6B8BDE8104000F0DCB8BDE870
:10A42000104000F001B9BDE8104000F018B902205A
:10A4300000F04CF82021052000F09EF800210120BA
:10A44000BDE8104018E010B50C4622469821FFF7F1
:10A4500001FE21460120FFF7A8FE30210120FFF771
:10A460002EFE1448032180F8201014488168091B2F
:10A4700081600021017310BD10B50C460F4B1249CD
:10A48000196018730D2298211846FFF7E3FD0D217E
:10A490000120FFF78AFE0748052180F8201044B10B
:10A4A000042180F8201030210120BDE81040FFF782
:10A4B00006BE10BD4831002008310020C031002008
:10A4C00055534243283200205553425380B518B1AA
:10A4D000022807D00AD301BD10210120BDE80440A5
:10A4E000FFF7EDBD10210120FFF7E9FD4FF480518A
:10A4F0000220BDE80440FFF7F3BD00007449087C6A
:10A50000C00702D57348052105E00FF2E410C97CAD
:10A51000252928BF2421FFF796BF6F48002181809D
:10A52000022181710021C1714172022181720021D9
:10A53000C1720C21FFF787BF6848002101800F21FD
:10A540008170FF21C1700021818002218171002171
:10A55000C1710821FFF777BF04216148FFF773BF7E
:10A5600008216048FFF76FBF5948C17C132928BFF5
:10A5700012215D48FFF767BF5B4A90701173704707
:10A5800069E070B504460D46584E3078C0B92A4689
:10A590002146282000F076F8C8B14D48007B00061F
:10A5A00003D50220307029460CE00220FFF78EFF11
:10A5B00000F00EF801210120BDE87040FFF75CBFFC
:10A5C000022804D12046BDE87040FEF706BA70BDEF
:10A5D00024210520D0E710B5444C2278EAB90A4678
:10A5E00001462A2000F04EF8E8B13948007B000609
:10A5F00008D4012020704FF440510220BDE81040E3
:10A60000FFF76EBD0020FFF761FFFFF7E1FF0021BC
:10A610000120BDE81040FFF72FBF012A04BFBDE8AD
:10A620001040FEF72ABA10BD80B52948816829B9C3
:10A63000007C400702D40121002006E00220FFF741
:10A6400045FFFFF7C5FF00210120FFE7BDE80440FB
:10A65000FFF712BF00BF01210020FFF70DBF80B53B
:10A660001B48816809B9002004E0007B00064CBF4C
:10A6700000200220FFF72AFF2021FFF7AAFF002178
:10A680000120E3E780B55118B1F5805F09D92A2888
:10A6900004BF0220FFF71AFF0020FFF717FF212158
:10A6A0000BE00B498968B1EB422F0ED02A280CBF72
:10A6B00002200020FFF70AFF2421FFF78AFF002174
:10A6C0000120FFF7D9FE002002BD012002BD0000DD
:10A6D000483100200C320020A00800201432002055
:10A6E000C8080020BC080020500800206831002065
:10A6F00000800202200000004D696E692044534F23
:10A700004469736B2020202020202020202020203E
:10A710002020202010B5DFF8884700B92BE000F09A
:10A7200096F80068804720680A3010BD80B5DFF8D1
:10A7300070070068C178DFF86C2752788A420CD322
:10A740008278002A04BF8288002A06D1817200F034
:10A750007EF840688047002002BD022002BD10B58F
:10A76000DFF83C4700B906E000F071F880688047E8
:10A7700020680C3010BD206801210182002010BD2E
:10A7800010B5DFF81C472068C1784079DFF818273A
:10A7900012689269904721688A7A92B1002804BFB2
:10A7A000087900280DD1887858B900F050F8C068B1
:10A7B000804720684179C1722068C1780173002008
:10A7C00010BD022010BD1CB5DFF8D416096810B901
:10A7D0000220088239E0DFF8D44600202080087883
:10A7E00000227F23184215D1487A81064CBF42F0DF
:10A7F000020102F0FD0121702178400654BF01F0F2
:10A80000FE0041F00100207000F021F8006980474F
:10A81000204616BD00F07F03012BF9D000F07F0029
:10A82000022812D1487900F00F0142F0010200F035
:10A8300088FA05D500F030001028E5D12270E3E752
:10A8400000F44050B0F5805FF7E7002016BDDFF858
:10A85000600600687047F8B5DFF8440600680178C4
:10A8600011F07F0104D1417A01F0DF0141724FE024
:10A87000022901BF41880029017900294AD1417983
:10A8800021F08005DFF82C460A0654F825204CBF3D
:10A8900002F0300202F44052DFF808361B789D4285
:10A8A00038D2002A1CBF807A002833D0080654F81A
:10A8B00025000BD500F03000102825D12846FFF7E1
:10A8C00053FC30212846FFF7FAFB1DE000F440500E
:10A8D000B0F5805F18D148F280064BF68F7745B906
:10A8E00000F0BDFA2068384080F4405030432060CA
:10A8F0000AE02846FFF726FC54F82500384080F48B
:10A900004050304344F82500FFF7A1FF40698047DD
:10A910000020F2BD0220F2BD38B5DFF884050268E0
:10A92000537923F08000DFF88C151C0651F8204085
:10A930004CBF04F0300404F44054DFF868552D781F
:10A94000A84206D2558825B9002C1CBF927A002A4D
:10A9500001D1022032BD48F280021B0651F820309E
:10A9600005D548F6BF74234083F0100304E04BF68E
:10A970008F74234083F480531A4341F82020FFF75B
:10A9800066FF80698047002032BD80B5DFF8100582
:10A990000068417A41F020014172FFF758FFC06919
:10A9A0008047002002BDDFF8F8241268538A20B9DE
:10A9B0008888C01A108200207047086818187047ED
:10A9C000F8B5DFF8DC54286800F110042688A16887
:10A9D000080018BF002E14D0A088864288BF064603
:10A9E0003046884707462088801B208060883018C2
:10A9F00060800020FFF7D2FB324601463846FFF761
:10AA00003EFBDFF8B464208850B1DFF8B0044FF4A7
:10AA10004051018000210020FFF7C7FB302030802B
:10AA200028682188A288914228BF032101D211B150
:10AA300005210172F1BD06210172DFF8840400686E
:10AA400080B2DFF88014002241F8102030203080DE
:10AA5000F1BD2DE9F843DFF84844206800F1100605
:10AA60003188DFF85454002904BF007A042816D135
:10AA7000DFF85404017801290DD1DFF84414096886
:10AA800089B2DFF84024002342F8113030212980B8
:10AA9000042703702CE007271020288028E0B6F850
:10AAA0000480884505D30427414588BF4146884630
:10AAB00000E002274046B168884781460020FFF742
:10AAC0006CFB424601464846FFF7C4FA4146002067
:10AAD000FFF76BFB3088A0EB0800308070884044A3
:10AAE000708030202880DFF8D4034FF4405101807B
:10AAF00020680772BDE8F18338B5DFF8A443206809
:10AB0000457801787F22114238D1092D02D1FFF713
:10AB10000DFE47E0052D1BD1C17880294FD28178E9
:10AB2000002901BF81880029807A002847D10620AA
:10AB3000DFF88C13096889B2DFF88823002342F814
:10AB40001130DFF8741330220A802168087231BD99
:10AB5000032D08D1C178012904BF8088002823D1A2
:10AB6000FFF713FF1EE0012D04BFC17801291BD19F
:10AB70008188C9B9407A80060DD415E001F07F00C4
:10AB8000012804D10B2D0FD1FFF7FAFD0AE00228AE
:10AB90000AD1012D02D1FFF75EFE03E0032D03D1A0
:10ABA000FFF7BAFE0028C2D02846BF4909684969A4
:10ABB0008847032808BF0920C7D00028B7D008203D
:10ABC000C3E738B5B64D28684178B74C062913D18C
:10ABD00001787F2211422AD18078012802D1206891
:10ABE000C16968E0022802D12068016A63E0032895
:10ABF0001DD12068416A5EE000293DD141880029CD
:10AC000004BFC188022912D1017981B901787F225C
:10AC1000114204BF8288002A2CD001F07F02012A51
:10AC200010D100F089F810B92868807A10BB286824
:10AC30004078216809698847032845D12868092197
:10AC4000017231BD01F07F010229F0D1407900F09D
:10AC50000F0100F0700200F074F84CBF00F03000FB
:10AC600000F440508F4B1B789942E0D2002ADED18D
:10AC70000028DCD095491EE0082905D100787F2105
:10AC80000842D4D1924916E00A2902BF017801F0A6
:10AC90007F010129CBD1817A0029C8D041880029C0
:10ACA00001BF01790029C1880129C0D100F044F811
:10ACB0000028BCD187490800B9D028680022428208
:10ACC000816100208847002029680A8A4FF6FF73B7
:10ACD0009A4208BF092004D0022818BF002A02D1D6
:10ACE0000820087231BD087800061ED5C88800907B
:10ACF0002368009C944202D2009808820FE08242AE
:10AD00000DD293F82C00704C824238BF002005D33E
:10AD100092FBF0F500FB152008B90120207093F894
:10AD20002C008882BDE8314093E603200872634816
:10AD30004FF44051018031BD002140792268926971
:10AD400010475C4B000653F82100704738B55C484B
:10AD5000006880B2604931F81000400000F1804086
:10AD600000F5C0404E4C21680A7A092A14D010F828
:10AD7000012B0A70216810F8012B4A70851C35F8E8
:10AD8000040BFFF763FA216848802888FFF75EFA12
:10AD900021688880A888C880206801210172206805
:10ADA000C08810B9FFF7A8FE01E0FFF70AFFBDE871
:10ADB00031403EE010B53A4C2068017A022918BFB4
:10ADC000042904D1FFF745FE2068007A14E0062923
:10ADD00011D14178052902BF01787F22114206D1A5
:10ADE000C07800F042F8FFF732FD006A80472E4835
:10ADF000006880688047082017E010B5284C20685C
:10AE0000007A022818BF04280ED0032818BF05288E
:10AE100004D1FFF7D5FD2068007A06E0072803D1AA
:10AE200021480068C0688047082021680872BDE892
:10AE3000104080B500F013F819480068017A08291D
:10AE400006D11E494FF480520A801B4910220A8005
:10AE5000007A092801D1012002BD002002BD1F484F
:10AE600090F82C100020FFF7A7B970B50D490978AC
:10AE70000022104B48F68F760BE0D4B253F82450E2
:10AE80003540254345F4004545F0800543F82450FE
:10AE9000521C8A42F1D340F080001149086070BD15
:10AEA00090310020C408002094310020303200206E
:10AEB00098310020005C00403632002034320020FF
:10AEC000505C0040046000403E320020C7A70008EC
:10AED00015A700085FA700080860004014070020BD
:10AEE0004C5C00407047000080B500F0F8F88B48DB
:10AEF00000680021817200F031F989480021416029
:10AF00004FF40441874A11800160874800210160A5
:10AF100001BD10B5854800218172804800688449D0
:10AF2000C97941720020FFF7B9F84FF40071002091
:10AF3000FFF7BBF820210020FFF7C1F818210020FF
:10AF4000FFF724F97B4C00F042F858210020FFF76E
:10AF50001CF90020FFF7E7F80020FFF7D8F80021E0
:10AF60000120FFF7A2F898210120FFF70EF9202118
:10AF70000120FFF7A4F800210120FFF7B1F800211C
:10AF80000220FFF792F8D8210220FFF7FFF894F88B
:10AF90002C100220FFF710F94FF440510220FFF768
:10AFA0009FF800210220FFF78AF800F010F8002037
:10AFB000FFF7ADF80020FFF758FF5B480121016063
:10AFC0005D485E4901605E480021017010BD94F843
:10AFD0002C100020FFF7F0B850480068807A00B9C4
:10AFE000704780B55048052101600120FFF7BCF88B
:10AFF0000220FFF7A7F852480021017001BD4E481A
:10B0000000684E4988421CBF0220FFF75FBA7047B4
:10B0100045480421016070477047704780B53F493B
:10B0200009680A7802F07F02212A08BFFE280BD1A6
:10B030004888002801BF88880028C888012803D1D3
:10B040000FF28900020001D1022002BD88610020B8
:10B05000488200F03BF8002002BD80B52F49096806
:10B060000A7802F07F02212A08BFFF2815D14888FC
:10B07000002804BF888800280FD1C88868B901203B
:10B08000FFF772F80220FFF75DF82B482B490160AB
:10B090002B4800210170002002BD022002BD0029C2
:10B0A0000CBF0028022070472649FFF77CBC2649C8
:10B0B000FFF779BC19490968C978062901DB002026
:10B0C0007047224A02EBC101FFF76DBC28B9134853
:10B0D000006801210182002070471D4870471D480B
:10B0E00001684268806801B9704710B51A4B9970C1
:10B0F0000C0A1C710C0C9C71090E19729A72110ABF
:10B100001973110C9973110E19749874010A197539
:10B11000010C9975000E187610BD000090310020CA
:10B12000405C00403A3200202C3200207431002074
:10B13000CCB8000814070020483100205553424382
:10B1400068310020AC080020B408002070070020FF
:10B1500028320020E8F7FF1FBC0700200648012125
:10B1600001600021016041604FF4E051034A118009
:10B17000FFE7016000207047405C00403A32002049
:10B1800053746254656D7000576B54656D700000A8
:10B19000536C7054696D650052617465645F500052
:10B1A00054656D70537470004F6666566F6C740012
:10B1B00054656D700000000048616E64000000007E
:10B1C0005A65726F505F416400000000506F7274E6
:10B1D00061626C650000000053746254656D703DDF
:10B1E00032303000576B54656D703D3330300000A5
:10B1F000536C7054696D653D31383000526174652F
:10B20000645F503D3138000054656D705374703D7B
:10B21000313000004F6666566F6C743D313300006C
:10B2200054656D703D30000048616E643D30000033
:10B230005A65726F505F41643D313032000000004A
:10B24000506F727461626C653D31000020202023D4
:10B25000283130307E343030290D0A002020202063
:10B2600023283130307E343030290D0A00000000B0
:10B27000202020232836307E393939290D0A000054
:10B2800020202020232831367E3234290D0A000068
:10B29000202020202328317E3235290D0A0000008D
:10B2A0002020202023283130307E313230290D0AF1
:10B2B0000000000020202020202020202328303AD9
:10B2C000432C313A46290D0A00000000202020209E
:10B2D000202020202328303A4C6566742C313A52C5
:10B2E00069676874290D0A00202023446F206E6F5F
:10B2F00074206D6F64696679210D0A00202020207A
:10B300002328303A6E6F7420706F722C313A706F50
:10B3100072290D0A000000008168C26891420BD1B9
:10B3200007E002681168891853685B18C360083227
:10B330000260C2689142F4D04A1C8260087870476B
:10B340002DE9F04D88B000F10801039101684A0829
:10B35000039B03EBC202049200220592069200EBCB
:10B36000810101F10806406800F0010102914008E6
:10B3700006EBC00001900024154601E0AC4205D167
:10B380000198864202D108B0BDE8F08D00F077F850
:10B39000074617F0030803D100F071F800F1030825
:10B3A000381100900F2819D100F069F80F30009083
:10B3B00014E000F064F88246AC420DD10198864258
:10B3C00008BF00F05EF83468029800B14C44706821
:10B3D00005190836AC42F1D004F801ABB8F1010808
:10B3E000E7D100980028C9D000F049F88046B8108D
:10B3F00000F00300032804BF03A8FFF78DFF3746C2
:10B400002146AB4608EB002006E0801A083F796829
:10B410003A6801EB020B59463A688A1A8242F4D321
:10B42000404200EB010A4FF0000805E09DF81C00C7
:10B4300004F8010B08F101080098801C80459DD09C
:10B44000DA4507D157F804AB57F8040B00EB0A0BA9
:10B45000DA45F7D01AF8010B8DF81C00AC42E5D1A3
:10B460000198864208BF00F00CF83468029800B1D9
:10B470004C44706805190836AC42F1D0D6E703A8F1
:10B480004AE7012000F000B8C046C046024A110059
:10B490001820ABBEFBE700BF26000200576B5465C7
:10B4A0006D70200053746254656D7000536C70545D
:10B4B000696D6500506F77657220200054656D706E
:10B4C000537470004F6666566F6C740054656D70EF
:10B4D0002020200048616E6420202000536F757288
:10B4E000636500000000000000E018040404041874
:10B4F000E000000F3040404040300F0000000808DE
:10B50000FC0000000000000040407F4040000000C0
:10B510000078040404040488700000605048444229
:10B5200041407000003804048484C83000000038B2
:10B530004040404040211E00000080601008FE0096
:10B5400000000007040444447F4444000000FC045D
:10B5500084848404040000384141404040211E009E
:10B5600000C03088848484041800000F31404040BB
:10B5700040211E00001C04048444340C040000001C
:10B58000007E0100000000000070880404040488AC
:10B590007000001C2241414141221C0000F00804BF
:10B5A00004040418E000003041424242221907001E
:10B5B000000000000000000000000000000000008B
:10B5C000000000001C1CC030080404040830000007
:10B5D00007182040404020101C120C0202FE8282FC
:10B5E000E20200000000407F400003002DE9F84F18
:10B5F0000020ADF8000040F68F7848F60F7B48F247
:10B600008006444F444CDFF81491DFF814A14BF648
:10B61000BF7525E054F82010ADF80010BDF80010FB
:10B6200009040BD554F8201008EA010144F8201051
:10B630003C4901EB800050F8040C8047BDF8000045
:10B6400000060DD599F8000054F820100BEA01010E
:10B6500044F82010344901EB800050F8040C804776
:10B66000606CAAF80000000452D5BAF8000010F08F
:10B670000F0089F80000CDD120683880388800F0AC
:10B6800030007880388800F44050388020682840A6
:10B6900080F4005080F0200030432060BAF80000B1
:10B6A000C006206805D40BEA00002060FFF782FB8B
:10B6B00016E0ADF80000BDF80000000506D52068D2
:10B6C00008EA00002060FFF741FB09E0BDF8000038
:10B6D0000004C5D5206808EA00002060FFF78DFB54
:10B6E000206828403988C90448BF80F480503988D0
:10B6F000890448BF80F400507988C90648BF80F0AB
:10B7000010007988890648BF80F02000304320600F
:10B71000BDE8F18F34320020005C00403F32002051
:10B7200038320020F4070020D80700202E48016896
:10B7300041F00101016041682C4A114041600168FB
:10B740002B4A11400160016821F4802101604168A9
:10B7500021F4FE0141604FF41F0181600021026865
:10B7600042F4803202600268491C920302D4B1F5AF
:10B77000A06FF8D10168890330D51E490A6842F0EC
:10B7800010020A600A68920892000A600A6842F091
:10B7900002020A604168416041684160416841F4C9
:10B7A00080614160416821F47C114160416841F44D
:10B7B000E8114160016841F0807101600168890110
:10B7C000FCD54168890889004160416841F0020167
:10B7D0004160416801F00C010829FAD106484FF098
:10B7E0000061016070470000001002400000FFF897
:10B7F000FFFFF6FE0020024008ED00E0FCF785F8B0
:10B800004FF48040FCF7C8F8FCF765FAFCF7F1F854
:10B810000120FCF721FB0020FCF755F8C820FCF7BD
:10B8200047F80020FAF77BFF0020FCF715FB01200A
:10B83000FCF749F800F030F8FDF7A5FFFCF781F9B7
:10B84000FDF78BFFFDF755FFFAF762FFFCF79FFB53
:10B85000FCF7DEFEFCF727F8F8F77CFCFBF7BAFEF6
:10B86000FBF7E6FEFBF715F840F6B830FAF7C4FE32
:10B870004FF4167140F2DC50FCF7B4FAFCF7FDF916
:10B880000120FAF73DFDFAF736FDFDF7F6FEFAF76F
:10B89000C8FEFBF729F9F8E70448C06102210172EC
:10B8A00003490162034A426208680047743100207C
:10B8B0001407002098070020120100020000004039
:10B8C0008304205700020102030100000902200046
:10B8D000010100C0320904000002080650040705F7
:10B8E0008102400000070502024000000403090431
:10B8F0002603530054004D006900630072006F007E
:10B9000065006C0065006300740072006F006E00DB
:10B9100069006300730000002603530054004D00CB
:10B920003300320020004D006100730073002000DE
:10B93000530074006F007200610067006500000032
:10B9400010035300540020004D0061007300730089
:10B9500070B50D4C0D4D286820800D4E2088318823
:10B960000840400505D50B48406880474FF6FF303A
:10B970002860208831880840000444BFBDE870403A
:10B98000FFF734BE70BD000038320020445C004038
:10B990003A32002014070020FEF75EBCFEF77DBCA3
:10B9A0007047FEE7FEE7FEE7FEE770477047704727
:10B9B0007047FFF7CDBFFCF7C8B9FCF7E9B980B510
:10B9C0002020FEF777F928B12020FEF77EF9024803
:10B9D0000121017001BD00003C32002010B5074973
:10B9E00079441831064C7C44163404E0081D0A687A
:10B9F000511888470146A142F8D110BD0800000047
:10BA00003000000063B8FFFF74290000CC0800205C
:10BA1000000000002DF9FFFF0200000002000000FE
:10BA20006C0100000F02000000000020CC080000A4
:10BA300000F009F8002801D0FFF7D0FF0020FFF741
:10BA4000DDFE00F002F80120704700F001B80000B0
:10BA500007463846FFF718FDFBE70000014880471E
:10BA6000014800472DB700086DBA0008C046C0461F
:10BA7000C046C046FFF7DCFFFFF792BFFFF791BF5C
:10BA8000FFF790BFFFF78FBFFFF78EBFFFF78DBFA8
:10BA9000FFF78CBFFFF78BBFFFF78ABFFFF7FEBF33
:10BAA000FFF7FEBFFFF7FEBFFFF7FEBFFFF7FEBFCA
:10BAB000FFF7FEBFFFF7FEBFFFF7FEBFFFF7FEBFBA
:10BAC000FFF7FEBFFFF7FEBFFFF7FEBFFFF7FEBFAA
:10BAD000FFF7FEBFFFF7FEBFFFF7FEBFFFF7FEBF9A
:10BAE000FFF7FEBFFCF79FB9FFF7FEBFFFF761BF8F
:10BAF000FFF7FEBFFFF7FEBFFFF761BFFFF7FEBF17
:10BB0000FFF7FEBFFFF7FEBFFFF7FEBFFFF753BF14
:10BB1000FFF753BFFFF7FEBFFFF7FEBFFFF7FEBF04
:10BB2000FFF7FEBFFFF7FEBFFFF7FEBFFFF7FEBF49
:10BB3000FFF7FEBFFFF7FEBFFFF7FEBFFFF7FEBF39
:10BB4000FFF7FEBFFFF7FEBFFFF7FEBFFFF7FEBF29
:10BB5000FFF7FEBFFFF7FEBFFFF7FEBFFFF7FEBF19
:10BB6000FFF7FEBFFFF7FEBFFFF7FEBFFFF7FEBF09
:10BB7000FFF7FEBFFFF7FEBFFFF7FEBFFFF7FEBFF9
:10BB8000FFF7FEBFFFF7FEBFFFF7FEBFF2FF0001AA
:10BB9000F1DE01100380B1000888041290041298AD
:10BBA0000412A00412A80412B00412B80412C004B3
:10BBB00012CC242002040C74802F2001740C043752
:10BBC0005003031C601C0342124001211C1003009F
:10BBD000001F2242012322131730014040C01B32B4
:10BBE000C00C70027F41404074F001016060000CA5
:10BBF0002378040133887821E005504844424140CD
:10BC000070ADA1391001E018083010010818E07873
:10BC100010010F302085300120300F867001080898
:10BC2000FC6B117AF401FF404040F5F1FF01F1AEE9
:10BC3000011A10E91AA0FC1EE89203D2640C500B02
:10BC40003C86010070170000B80B0000182C120190
:10BC50003012FA0C520A044382002C520104F20EF4
:10BC6000000CF0071E601D00004808000064A8F6E4
:10BC700046330010034CB200085C041270041280BA
:10BC80000412900412A00412B40412CC0412E804AA
:10BC900012FC081ED8CC0412E40412F00412FC0CAE
:10BCA00012083812143C1220401228441230481254
:10BCB000402C100BE9AE000813AF000819B00008C3
:10BCC0001B04121D04125B04129F0412A90412AF7C
:10BCD0000412B51C3D6104157010039CB40008A447
:10BCE0000412AC0412B40412BC0412C40412CC0436
:10BCF00012D40412DC0452E4041FECB84C05158085
:10BD000012F0081626144318B9082003BC070020B7
:10BD10001A50111025D012E58412D98483E5AE049F
:10BD200092FF1012119C14051A03530054004D5831
:10BD3000B403320031003014F0040999B90008E569
:10BD4000AE04F2069D207815AED552A80FC0D300E0
:10BD500040A08D14DA028133D9F1DB30A4A6AF0103
:10BD60005A66303A3C0DF600018C5DB405FA0B0AB8
:10BD7000ACA110495CF3010A004A3C01000088496B
:10BD800006456816022416B83416121C16CC3C223E
:0CBD9000201A42066D1A03D12D8D06000A
:040000050800BA6DC8
:00000001FF
